:100200004F726967696E616C2046696C653A20704F
:10021000726F6A6563742E6865780D0A4F75747025
:10022000757420446174653A20323030392F30378C
:100230002F30380D0A4F75747075742046696C65DF
:100240003A206B6C39372E6865780000000000009A
:10025000000000000000000000000000000000009E
:10026000000000000000000000000000000000008E
:100270000000000000000000000000000000007C02
:108143000D0A0D0A205B4B4C39375D0D0A0D0A00F1
:108153000D0A0D0A00557365204B4C3937432049EE
:108163004F20446566696E650D0A005365742041AE
:1081730064383139782053776974636820526567AE
:1081830069737465720D0A00536574204164383154
:10819300397820537769746368205265676973740B
:1081A300657220446F6E650D0A00416C6C204F753B
:1081B3007470757420456E61626C650D0A00416CC4
:1081C3006C204F757470757420446973616C650D10
:1081D3000A0052656D6F746520696E2052554E20FA
:1081E3006D6F64650D0A0052656D6F746520506193
:1081F300737320434841206B65790D0A0052656D06
:108203006F7465205061737320434842206B657916
:108213000D0A0052656D6F746520506173732043BE
:108223004843206B65790D0A0052656D6F746520B4
:108233005061737320434844206B65790D0A000233
:108243008000400010002000010002000400000232
:0F8253008000400010002000010002000400081D
:108E4B0041FA780041F9040041F90B0041F90300A4
:0C8E5B0041F9010041F9020041FA8B00CE
:108FD00074FF90F90CF07B017AF9790C90FD9AE41A
:108FE000F0A304F0227401F0A374F9F0742EA3F03E
:108FF000A37401F0A32290FDABE0FF7401A8070861
:10900000227B0190FD9AF0A304F0E4FD7F9422906E
:10901000FDAAE075F021A42412F582E5F034F9F5FB
:1090200083E022EF75F021A4240DF974F935F0FAEC
:109030007B01227401F0A374F9F0A3744F2290FD18
:10904000AAE0FFC32290FDAAE004F022A4240DF5BB
:1090500082E5F034F9F583E0227B017AF979012287
:109060007401F0A374F9F0A3740DF022A3F07B0156
:109070007AF9790722A3F07B017AF979092290F92C
:1090800003E090F9012290F903E0FF90F901E0225A
:103DA500E490FDAAF0A3F0A374FFF0A3F0E4A3F060
:103DB500A3F07F0512B5E5E4F5207DFF7F05127AB6
:103DC500B87B027DFF7F051269A77D1E7F02127AEF
:103DD500B87B027D1E7F021269A77D037F061279DB
:103DE500517B027D0312431E7D017F0A1269A7E400
:103DF500FB7D037F0C1269A7E4FB7D0F7F01126930
:103E0500A7E4F5F1FB7D0412431E7D087F061269C8
:103E1500A7D2AF75FF387BFF7AB479B412B5F1E458
:103E2500FF12ABC77D017F407E021294A97BFF7A0A
:103E350081794312A71E7BFF7A02790012A71E7BA8
:103E4500FF7A81795312A71E7BFF7AB679577F03D4
:103E550012B6137B007C077DD012006E7BFF7A8142
:103E6500795812A71E90FDFB74FFF0A37482F0A38E
:103E75007452F07B017AF8790012AE157D0C7F0B38
:103E8500127AB87B017D0C7F0B1269A77D017F0833
:103E9500127AB87B027D017F081269A71298597DB5
:103EA500017F081279517F0112B5E57B017AF97915
:103EB5000DE4FD12837E7AF9792E7DB41242FE7AE5
:103EC500F9794F7DB912837E7AF979707DE01242D6
:103ED500FE7AF979917DE512837E7AF979B27DEAE8
:103EE50012430E7AF979D37DEF12837E7AF979F44C
:103EF5007DD012430E7AFA79157DD512837E7B012A
:103F05007AFA79367DDA12837E7B017AFA79577DE2
:103F1500DF12837E7B017AF979057D701295EA12AD
:103F2500906E7D7E1295EA1290777D7C1295EA7AE5
:103F3500FA79797D601243067AFA797B7DE0129FE2
:103F4500CE7AFA797D7DE21243067AFA797F7DE4AD
:103F5500129FCE7AFA79817DE61243267AFA798321
:103F65007DE8129FCE7AFA79857DEA1243267AFAA0
:103F750079877DEC129FCE7B017AFA79897DEE12E5
:103F85009FCE90FCF6129060A3128FE5129037F049
:103F95007B017AF9790512871490FCF6128FE57486
:103FA500F9F07470128FEE74F9F0749112906C122E
:103FB500871490FD02128FE574F9F0A374B2128F85
:103FC500EF74F9F074D312906C128F0F90FCF61207
:103FD5009033128FEF74F9F0A374F4128FEF74FA23
:103FE500F0741512907512871490FD021290331219
:103FF5008FEF74FAF0A37436128FEF74FAF07457DA
:10400500129075128F0F90FE011290607B017AFA63
:10401500797912B503E490FDAAF012903E94085008
:104025003FEF75F002A4247BF974FA35F0FA7B01B1
:10403500C003C002C0017E007C007D211219FB7403
:10404500702FF974F93EFA90FE01EBF0A3EAF0A3A4
:10405500E9F0D001D002D00312B50312904580BA21
:10406500E4FFFE12B45DEFD39403E4400690FE3600
:10407500F0800AFFFE12B45D90FE36EFF090FE363A
:104085007401F07BFF7A81796E12A71E7440128F3E
:10409500D2E4FD7F94128B29128FD6FD7F94128B6B
:1040A5002990F90C7401F0FB128FD87D107F9412C2
:1040B5008B29128FD07D117F94128B29128FD67D7B
:1040C500127F94128B29128FD07D137F94128B2926
:1040D500128FD67D147F94128B2990F90C740312DC
:1040E5008FD57D207F94128B297BFF7A81798B1266
:1040F500A71E90F9017443F01243167D027F021248
:104105007AB812A7B82008030242F8C20890FDAA9F
:104115007403F0E4A3F012903E940B40030241C8EF
:1041250075F021EF12904CFB703912900FFC30E4C2
:104135000C128FF68002C333D8FC0241A7EC30E5A0
:104145001790FA78E075F01484E5F0706C128FF62C
:104155008002C333D8FC8039128FF68002C333D86E
:10416500FC8050EB6405600E90FDAAE075F021120D
:10417500904C640C703412900F30E61D90FA78E084
:1041850075F02884E5F07031128FF68002C333D8BC
:10419500FCFD7F05126C838020128FF68002C333ED
:1041A500D8FCFD7F05127AB8800F128FF68002C306
:1041B50033D8FCFD7F05127951129045A3E004F038
:1041C50002411B90FA78E004F0C394C84002E4F081
:1041D5007B017AF9790D1237F190FDAA7401F0127D
:1041E500903E9403500B1290231257DB129045809A
:1041F500EE90FDAA7403F012903E940B500B1290B2
:10420500231223A112904580EEE520B4FF0D7D0217
:104215007F061279517D1E7F02804C7D027F06123A
:104225007AB890F901E0FCB443071243167D028089
:104235002FECB4420B7D1E7F021279517D04802044
:1042450090F901E0FCB4410B7D1E7F021279517D8E
:1042550008800DEC7D1E7F02B4400C1279517D1053
:104265007F02127AB8800312795190FDACE025E007
:10427500F0E0FE7D047F061297C0EF60047F0180A9
:10428500027F00EE4FFF90FDACF0BF7F0EE520B43E
:10429500FF047F1D80027F0212801690FDADE02590
:1042A500E0F0E0FE7D087F061297C0EF60047F0115
:1042B50080027F00EE4FFF90FDADF0BF7F057F04CC
:1042C50012801630090AC2097F0112B11812801630
:1042D50012432E200D0302410A90FA8BE0FF04F0F1
:1042E500EFD39464500302410AC20D7F1D1280165C
:1042F50002410A43870102410A7B0112837E7B0149
:10430500227B01129FCE7B01227B0112837E7B01E2
:10431500227D1E7F02127951227F061269A7E4FBD6
:09432500227B01129FCE7B0122D4
:10801600E490FEEEF0EF14700302810814602F1452
:10802600700302811E1470030280DD24F2602A248C
:10803600F870030280FD24FE7003028113146003AE
:108046000281307BFF7A8179AD12A71E804C7BFFBF
:108056007A8179C112A71E8004E520703D7520FF44
:108066007B017AF9797012B5FD7AF9799112B5FD2D
:108076007AF979B212B5FD7AF979D312B5FD7AF9A2
:1080860079F412B5FD7AFA791512B5FD7AFA7936D0
:1080960012B5FD7AFA795702B5FDE4F5207B017A2F
:1080A600F9797012B6087AF9799112B6087AF979DF
:1080B600B212B6087AF979D312B6087AF979F412B7
:1080C600B6087AFA791512B6087AFA793612B60827
:1080D6007AFA795702B6087A8179D5128131E09019
:1080E600F903F064406005E014F0800690F903742B
:1080F60043F012907E802F7A8179EA12813174439F
:1081060080247A82790012813A744280197A8279BF
:108116001612813A7441800E7BFF7A82792C12A75F
:108126001E90F9017440F012A7B8227BFF12A71E19
:0D81360090F901227BFF12A71E90F9012293
:10A95F00129086FD6F6039EDB443047E08801AEDC6
:10A96F00B442047E048012EDB441047E02800AEDED
:10A97F00B440047E018002E4FE7D0F7F011297C078
:10A98F0090F904EFF05EFE700712907EF012A7B8F8
:01A99F002295
:10A9A0001290866F6039EFB440047E01801AEFB4D4
:10A9B00041047E028012EFB442047E04800AEFB4A8
:10A9C00043047E088002E4FE7D0F7F011297C09051
:10A9D000F904EFF05EFE600712907EF012A7B82235
:10A7B800E490FEEFF0F07AFE79EF129001128B2907
:10A7C8007B017AFE79EF128FDC12A7FC7F0112B5AC
:10A7D800E5129059128FDCE412A7FC129059128FDF
:10A7E800DCFD7F94128B297F02128016E490FA8B8D
:0BA7F800F0D20D22FD7F94128B29226D
:10AA5E00E490FEF0F0F07AFE79F0129001128B295C
:10AA6E007B017AFE79F0128FDCFD7F94128B297FA9
:10AA7E000112B5E5129059128FDCE4FD7F94128B12
:0DAA8E0029129059128FDCFD7F94028B2954
:10ADB000E490FEF1F0F07B017AFE79F1129003123B
:10ADC0008B297B017AFE79F1128FDCFD7F94128B47
:10ADD000297F0112B5E57F02128016E490FA8BF00C
:03ADE000D20D226F
:10B4B400AE07E4FF12B118BF0109EE7006EDB41037
:04B4C40002D2092285
:03B65700D20822F4
:104881000000000000000000000000000000000027
:104891000000D60980A020E02D101060A2000403C2
:1048A100000000188C0AD08A20E02D10103E9600DE
:1048B1000403000000188C0AD08A20E02D10103E5D
:1048C1009600100900000018011D007251D01E2031
:1048D1006E28550010090000001E011D8018711C72
:1048E1001620582C250010090000009E8C0AA014E7
:1048F10051F01600267C43000403000000988C0A46
:10490100A01451F01600267C430010090000009805
:104911008C0AA01451F01600267C43000403000009
:1049210000188C0AA01451F01600267C43001009CF
:104931000000001818154028B2F016004CF843008A
:1049410004030000009818154028B2F016004CF836
:10495100430010090000009818154028B2F0160015
:104961004CF8430004030000001818154028B2F069
:1049710016004CF843001009000000181815A01487
:1049810051E02D10207C960004030000001818153A
:10499100A01451E02D10207C960010090000001891
:1049A100023A801871382D40582C4500100900003A
:1049B100001E8C0AD090204031200C405500040389
:1049C100000000188C0AD090204031200C40550086
:1049D100100900000018011D00BC52D01E20B8288B
:1049E100554010090000001E011D80D0721C1620C8
:1049F100102C258010090000009E8C0AA020512057
:104A01001810187E23000403000000988C0AA020CF
:104A110051201810187E23001009000000988C0AFC
:104A2100A02051201810187E230004030000001854
:104A31008C0AA02051201810187E230010090000B4
:104A4100001818154040B220181030FC2300040350
:104A51000000009818154040B220181030FC2300C7
:104A610010090000009818154040B220181030FCC1
:104A7100230004030000001818154040B22018104C
:104A810030FC23001009000000181815A020514027
:104A910031201880550004030000001E1815A020C5
:104AA100514031201880550010090000001E023AC3
:104AB10080D072382D40102C458010090000001E56
:104AC100011D803E73382D407E2C45801009000069
:104AD100001E011D80D072382D40102C4580100918
:104AE1000000001E011D80D072382D40102C458021
:104AF10010090000001E3B2A4028B2E02D1060F88A
:104B010096000403000000183B2A4028B2E02D1053
:104B110060F89600100900000018302A4040B240A9
:104B2100312030005510040300000018302A4040A5
:104B3100B240312030005510100900000018201C2F
:104B41008080711C552020A8750410090000009A6E
:104B5100023A80D0721C1620102C2580100900000A
:104B6100009E023A00BC52D01E20B82855401009C0
:104B71000000001E1815D090204031200C40550037
:104B81000403000000181815D090204031200C407B
:104B910055001009000000181815D0902020181099
:104BA100187E23000403000000981815D0902020DF
:104BB1001810187E2300100900000098023A80188E
:104BC100711C1620582C250010090000009E023A85
:104BD100007251D01E206E28550010090000001EE1
:104BE1001D15D08A20E02D10103E96000403000010
:104BF10000181D15D08A20E02D10103E96001009D6
:104C0100000000181D15A01451F01600267C430069
:104C11000403000000981D15A01451F01600267C15
:104C21004300100900000098302AD0902040312024
:104C31000C405500040300000018302AD090204099
:104C410031200C405500100900000018302AA02026
:104C510051201810187E2300040300000098302A08
:104C6100A02051201810187E230010090000009880
:104C71003B2AD08A20E02D10103E9600040300004C
:104C810000183B2AD08A20E02D10103E9600100912
:104C9100000000183B2AA01451F01600267C4300A6
:104CA1000403000000983B2AA01451F01600267C52
:104CB100430010090000009800FFFFFFFFFFFF0005
:104CC1001710010901000000000E010380734178F3
:104CD1002A7C119E59479B27105054000000010166
:104CE1000101010101010101010101010101011D97
:104CF100007251D01E206E28550010090000001EC0
:104D01008C0AD08A20E02D10103E9600040300008A
:104D11000018000000FC0045502D48444D492D521B
:104D2100580A2020000000FD003B3D0F2E08000A1C
:104D310020202020202001D402031D714A84051364
:104D410014010203111210230907078301000065F2
:104D5100030C001000023A801871382D40582C4580
:104D61000010090000001E011D8018711C1620583A
:104D71002C250010090000009E011D00BC52D01E10
:104D810020B828554010090000001E011D80D07276
:104D91001C1620102C258010090000009E8C0AD0C2
:104DA10090204031200C4055000403000000180001
:104DB100000000000000001E097F070F7F07170792
:104DC100503F06C04D02005706005F7E01677E001E
:068E670041FE3600C12FA0
:10530C0090FC97E0FBA3E0FAA3E02480F9E43AFADE
:10531C00EEFF7E0029F9EE3AFA12195FFD90FCAA15
:10532C00E0FBA3E0FAA3E0F990FCA5E0F58275831D
:10533C0000ED1219D9EF2481FFEE33FE90FC97E0BB
:10534C00FBA3E0FAA3E0F98F828E83121978FF9009
:10535C00FCA5E02401FDE433FC90FCAAE0FBA3E0F7
:10536C00FAA3E0F98D828C83EF1219D990FCA0E09E
:10537C0090FC972482FFE433FEE0FBA3E0FAA3E069
:10538C00222480F9E43AFA90FCA0E0FF7C0029F991
:10539C00EC3AFA12195F541FFEEF2E90FCA2F0901B
:1053AC00FC9FE004F0A3E004F090FC97A3E0FAA3C8
:1053BC00E02480F9E43AFA90FCA0E022E92480F998
:1053CC00E43AFAEE7E0029F9EE3AFA02195FFF9000
:1053DC00FE38E02FFF90FE37E03400FEE92FF9EAAB
:1053EC003EFA12195FFF22F9900082121978C3FF5E
:1053FC0090FCA0E0FE9F22F98D828C83021978F933
:10540C008F828E8302197890FCA4E0FF90FE37E027
:10541C00FCA3E0FDC39F7480F8EC6480982290FCA0
:10542C00A0541F04FFE02FF02290FC9FE02480FF8B
:10543C00E433FE90FC9A2290FCA0E0FE90FCA2EFDC
:10544C00541FFFEE2FF022FE04F0EE7C0029F9EC45
:10545C003AFAEF0219C790FD197401F0A374FCF02D
:10546C00A374A5F090FCADE0F9A3E0FAA3E090FDE5
:10547C001CC9F0A3EAF0A3E9F022F97F807E0012A8
:10548C00193990FC9E7401F022F99000821219785F
:10549C00FF90FC9FE0FE2290FCA4F9E0FE04F08E4D
:1054AC0082758300EF0219D9EE2480F582E433F57E
:1054BC0083121978FF54E02290FC9FE02480FDE4D5
:1054CC0033FC90FE38E02DFD90FE37E03CFC90FC68
:1054DC009A2290FE37E0FEA3E0FF22F9900083129F
:1054EC00197854C0440190FCA3F090FDB37401F002
:1054FC00A374FCF0A374A4F090FCA722FF90FE35DB
:10550C00E02FF090FE38E004F02204F0EE2480FD51
:10551C00E433FC90FC9A2290FCA4E0FFC390FE388C
:10552C00E09F7480F890FE37E064809822E490FE4F
:10553C0035F090FE37F0A3F022FF7C0029F9EC3A0D
:10554C00FA02195F90FE37E004F022900023F91262
:10555C001978FF90FC9A22FF90FCA5E02402FDE450
:10556C0033FC90FCAA22E429F9EA3401FA12195FFF
:10557C0054FE1219C790FC9722F9EF900001021902
:10558C00D990FCA0E004F0E0FF7E0090FE37EEF036
:10559C00A3EFF090FCA0F022F98D828C83EF02191E
:1055AC00D9FF04F07E00E92F22900002F91219783D
:1055BC00FF90FC9722EF541FFFEE2F90FCA1F022DE
:1055CC00541F04FF90FC9FE02FF02290FCA0740469
:1055DC00F022F990007E021978900001740C1219D7
:1055EC00D9E49000020219D990FCA2E0FF90FCA033
:1055FC00E02290FCA0E0FF7E0090FE37E0FCA3E0F0
:10560C00FD2FFFEE3CFE90FCA2E0FBD3EF9B7480E1
:10561C00F86E9822541FFF90FE38E02FF090FE3762
:10562C00E03400222400F9EA3401FA02195F541F15
:10563C00FEEF2E90FCA2F090FC9FE004F022547F31
:10564C00FFEE2480FDEC33FC90FC9A2290FC9FE052
:10565C00FF7E00ED2FFFEE3CFE90FCA1E0FDD3EFB2
:10566C009D74806E982290FC9FE02480FFE433FEB2
:10567C0090FE38E02FFF90FE37E03EFE90FC9A2221
:10568C0090FCA0E004F022FD7C00EF2DFDEC3EFC34
:10569C00E92DF9EA3CFA02195FF9EF9000020219C0
:1056AC00D990FC9F7404F02274802DF582E43CF5B3
:1056BC008302197890000374101219D9E490000435
:1056CC000219D92480F9E43AA801FCAD032290FC1C
:1056DC00A5F9E0F58275830022C39405EE648094ED
:1056EC00802290FC9FE02480FDE433CD2FFFED3E23
:1056FC00FE90FC9A22FF90FC9FE02482222FF582E0
:10570C00E43EF583021978F9900082021978F99039
:10571C00010002197890FCA5E02403F022F9900016
:10572C007E74010219D9C390FCA6E094052290FC6A
:10573C009FE0FF7E002480FDEE33FC22F9900001F7
:10574C00E41219D9900002E4222480F9E43AFA22F6
:10575C0090FE36E0640322FC8D82F583021978F901
:10576C00900023021978F9900024021978F990001E
:10577C0025021978F990003602197890FCA0E024E3
:10578C0003F02290FCA1E0FF90FC9FE0D39F2290BD
:10579C00FC9FE02403F022EF2481FFEE33FE90FC0B
:1057AC009A2290FE35E014F4FF90FC9722A3F0A30C
:1057BC00EBF0A322F8AC02AD03A3221219C790FCA4
:0F57CC00B022900037021978F912227B7E00225A
:10B04F0090FE6DEB12547E90FE6D125385F9EA4916
:10B05F004B601590FE6D1253851256304401121934
:09B06F00C744021219C7C22F22C6
:109A180090FE70EB12547E90FE701253851255DE44
:109A28006401707690FE37F0A37404F090FE701213
:109A38005385125713125417504F1256B454E064FA
:109A480060701F74811256B6640370321254DE249B
:109A58008212570A640C70267483125709701F7F8C
:109A6800012290FE70125385F990FE38E02480FFA1
:109A78001256298F82F583121978125620F0125542
:109A88000F70A9125550029A3490FE701253851225
:0D9A9800571312552740037F00227F002244
:10A1910090FE73EB12547E90FE731253851255DEBE
:10A1A100C39401404E90FE37E4F0A37404F090FE96
:10A1B1007312538512571312541750211256B4FBC0
:10A1C10054E0FFBF6008ED2480FFE43CFE22EB1267
:10A1D1005620F012550F70D612555080D190FE7353
:10A1E100125385125713FFC3ED9F7480F86C98408A
:07A1F100028000E4FEFF22E2
:10AE460074811219C7740212558774031255EE9055
:10AE5600000374111219D974121256C990000574A0
:10AE6600041219D990FDB3125385F974060219C755
:10AC6F0074091219C790000174071219D9740712C9
:10AC7F0056A790FD19125385F974031219C790FD49
:10AC8F001C125385F974011219C790FD1C125385BC
:06AC9F001257480219D90A
:10B42F0074031219C71255E51256C090FDB9125385
:07B43F0085F974050219C72D
:10A91C0090FD1FEB12547E90FD1F125385F8AC0274
:10A92C00AD037BFF7A4D79B97E007F1812193990EF
:10A93C00FD22125385F974181219C790FD25125374
:10A94C0085F9744F1219C790FD251253851257487B
:03A95C000219D904
:1002800090FC97EB12547EE490FC9EF07B0190FC76
:10029000A704F0A374FFF074801257B974FFF074D0
:1002A0009E1257B974FFF0A374CBF0A3EBF0A374C4
:1002B000FFF0A374CEF090FC97125385F9EA494BF6
:1002C0007002FF2290FE36E0640260030203C190D8
:1002D000FC9712538512571A20E0030217D31255C8
:1002E000721253851257C012538512548690FC9A8D
:1002F0001253851255DE640160030217D390FC97F8
:1003000012538512571A20E1030217D3E42912561B
:100310003254FD1219C790FC9A125385125755C0DA
:1003200003C002C00190FC971253851256CFD00132
:10033000D002D00312548790FC9DE030E0030217F6
:10034000D31255D790FC971253851253F3400302F2
:1003500017D31253C8FF54E064607053EF541FC3A7
:10036000940750030217D312568CE0FF2485FDEE4C
:1003700033FC90FC97A3E0FAA3E012569D548F1231
:1003800057C7125385F9900006121978FDC3941EC1
:10039000500280027D1EEF2486FFE43EFE90FC9713
:1003A000125385F98F828E83ED1219D90217D390DB
:1003B000FC971253851253BD1253D012542A0203D4
:1003C0004490FC9A1253851255DED3940140037F6A
:1003D000002290005A121978707890005B121978F8
:1003E000707090005C121978706890005D12197836
:1003F00064FD705E12553E1254DEC39412EE6480AA
:100400009480504E90FC9A125385F9EF245AFFE4E1
:100410003EFE8F82F58312197890FCA3F090FE388F
:10042000E0246CFD1256291257648F828E831219B4
:10043000D990FCA3E0FF90FE38E0246CFD12562911
:100440008D82F583EF1219D912550F70AA125550EB
:1004500080A590FC9712538512571A30E00F125561
:10046000721253851257C012538512548612575C6C
:10047000600302054E90FC97125385125557125394
:100480008512576B4F4421FF90FCA7125385F9EF5B
:1004900012557E12538590002412555A125385121C
:1004A00057724F4408FF90FCA71253851255859050
:1004B000FC97125385F990002512555B1253851253
:1004C00057794FFF90FCA71253851256A590FC9ABE
:1004D000125385F990006C12197860030206299076
:1004E000006D121978600302062990006E121978C7
:1004F000600302062990006F12197864FD60030200
:10050000062990FC97125385F990006C12197860B7
:100510000302060190006D12197860030206019033
:10052000006E121978702490006F12197864FD70B3
:100530001A90007512555B125385F99000751219C7
:1005400078D39F50030206290205FE02060190FCA3
:100550009712538512555712538512576B5F4421DA
:10056000FF90FCA7125385F9EF12557E125385F9BF
:1005700090002412555B1253851257725F4408FF96
:1005800090FCA712538512558590FC97125385F95C
:1005900090002512555B1253851257795FFF90FC2E
:1005A000A71253851256A590FC9A125385125780B4
:1005B00060771257CEFF607190FC971253851257E7
:1005C00080603E1257CEFE6038EFC39E50028031ED
:1005D00090FC97125385F990003712555B125385A2
:1005E000F91257CE6F704290FC97125385F9900024
:1005F0003612555B125385125780C39F502BE980EA
:100600000690FC9A1253852436F9E43AFAC003C0E6
:1006100002C00190FC9712538524361256D1D001A6
:10062000D002D0037F4812548990FC971253851250
:10063000576BFF90FCA7125385F912195FFE6F707C
:10064000219000011255B9125385125772B5071245
:1006500090FCA71253851255B51253851257796F26
:10066000600312548E90FC97125385F9900023EE8C
:100670001219D990FCA71253859000011255B81297
:100680005385F9900024EF1219D990FCA7125385D5
:100690001255B5125385F9900025EF1219D97E0035
:1006A0007F1E7D0090FCA71253851257D47F2D7DAD
:1006B0000090FCAA1253851257D47F037D0090FC52
:1006C000AD1253851257D47F0C7D0090FCB01253AD
:1006D00085F912227BE490FCA3F090FCA5F090FC3D
:1006E000A4F090FCA6F090FC971253851255DE649E
:1006F0000160030208FF90FC9A1253851255DE60D8
:10070000030208FF302F0302184D90FC9712538507
:10071000F9900083121978FF54C0440190FCA3F0B3
:100720006F600312548E12575C705B1255D790FCA9
:10073000971253851253F3506D1253C8FF54E0645F
:1007400040703112544312558D90FCA2E0D31253E5
:10075000FB505390FCA4E0C3941E501390FC9712DE
:1007600053851253C9FF90FCA71253851254A3124C
:10077000568C80D590FC971253851253BD1253D0DE
:1007800012542A02072E90FC97125385F990008488
:10079000121978541F6406600312548E1254F61214
:1007A0005385F912AE461255D790FC971253851215
:1007B00053F3504B1253C8FF54E06420702F12546F
:1007C0004312558D1255F4FED39F503390FCA5E093
:1007D000C3942D501212530C12540B125563125322
:1007E000851255A41257211257870207C490FC970F
:1007F0001253851253BD1253D012542A0207A91264
:1008000055D790FC971253851253F3506C1253C86E
:10081000FF54E06480705012544390FCA01253B215
:100820001255AD1253D3FF90FCAD125385F9EF1260
:10083000557E1253851253BDFF04F0E92F1253D396
:10084000FF90FCAD12538512558590FC971253858D
:100850001253BDFF04F0E92F1253D3FF90FCAD12E9
:1008600053851256A5801290FC971253851253BDE2
:100870001253D012542A0208021255D790FC971234
:1008800053851253F3504A1253C8FF54E06460700A
:100890002E12544312558D1255F4FED39F50DD1283
:1008A0005732501690FC971253851253C9FF90FC93
:1008B000B012538590FCA61254A612568C80D89084
:1008C000FC971253851253BD1253D012542A0208BA
:1008D0007C90FC971253851257C0125385F97E0005
:1008E0007F8012193990FC971253851257291254A0
:1008F0008E90FE36E06003021463D22F02146390E0
:10090000FC9A1253851255DE640160030214211211
:10091000553A1254DEC39480EE6480948050169051
:10092000FC9A125385F9748012570912550870E227
:1009300012555080DD90FE35E0604890FC971253D0
:100940008512563054FD12557E12538512572912C6
:10095000548E90FC9A1253851254E7125385F91263
:10096000AE4612546290FCAA1253851218531253C9
:1009700085F912B42F90FE36E06003021463D22F83
:10098000021463302F0302184D90FC971253851206
:10099000571A30E12BE42912563254FD1219C79030
:1009A000FC9A125385125755C003C002C00190FC37
:1009B000971253851256CFD001D002D0031254871C
:1009C00090FC9A125385F99000831255B912538501
:1009D000F9900083121978FE5F54F0444190FCA313
:1009E000F06E600312548E12575C6003020AC61246
:1009F00055D790FC971253851253F350411253C8A8
:100A0000FF54E064407025125443801B1255F4FEDD
:100A1000D39F50DE90FC971253851253C9FF90FC70
:100A2000A71253851254A312568C80E090FC9712A3
:100A300053851253BD1253D012542A0209F2125692
:100A4000AD90FC9A125385125495C39F4003020B3C
:100A5000D61254B46440705C90FCA112544B1256F0
:100A60004312578F50DBE412553E12541350241298
:100A7000543512538512540B547FFF90FCA7125328
:100A800085125403547F6F600A12550F70DC1255A3
:100A90005080D712552340161254351253851254E4
:100AA0000BFF90FCA71253851254A312548E1257B9
:100AB0009B020A6112543512538512540B90FC9F0D
:100AC00012542D020A411255D790FC9712538512E9
:100AD00053F34003020BD61253C854E06440600342
:100AE000020BC41256AD90FC9A125385125495C352
:100AF0009F4003020BD61254B464406003020BB54E
:100B00001255C190FC971253851253BD12554512D0
:100B1000563AA3E004F090FC9FE0FF90FE37E4F02B
:100B2000A3EFF01255F4D39F4003020BD690FE378B
:100B3000A3E090FC9FF090FCA1E012549CD39F5046
:100B40004190FC971253851253BD12554612564AD6
:100B5000125385125403FE547F6F702090FCA4E062
:100B6000C3941E501790FC971253851253BD125513
:100B7000464EFF90FCA71253851254A3125643020F
:100B80000B3690FCA4E0FF602390FC971253851273
:100B900053BD125546FEEF24FFFDEC34FFFC90FCE4
:100BA000A71253851254036E6005800012548E12F2
:100BB000568C020B2312543512538512540B1255C6
:100BC000CC020AE690FC971253851253BD1253D003
:100BD00012542A020AC990FE36E0FF64016008EF51
:100BE00064036003020EC01255D790FC9712538520
:100BF0001253F350421253C8FF54E064207026127F
:100C0000544312568C1255F4FED39F50DD12530CF0
:100C100012540B1255631253851255A41257211208
:100C20005787020C0590FC971253851253BD12533F
:100C3000D012542A020BEA1256AD90FC9A12538538
:100C4000125495C39F4003020DF91254B4642060FE
:100C500003020DEA1255C112564312578F50DBE4BE
:100C600012553E90FCA51254164003020D8E1254EC
:100C70003512538512540B5478FF90FCAA125385F9
:100C8000125403FE54786F6003020D8190FC9FE0C4
:100C90001255191253851254035407FFEE5407FEE0
:100CA000D39F4004AF06800090FC9FE012551912BC
:100CB000538512540354784FFF90FCAA125385F9C0
:100CC00090FE37E0FCA3E0FDF5828C83EF1219D98A
:100CD00090FC9FE0248112543B12538512540BFF69
:100CE00090FCAA125385F9ED2401FDE43C125763F0
:100CF0004F8D828C831219D91254DEF5828E8312A5
:100D000019785478FDBD013690FCAA125385F9EF8D
:100D10002402FFE43EFEE92FF9EA3EFAC003C002D6
:100D2000C00112195F12570112551B12538512543C
:100D3000034FD001D002D0031219C7020D8E90FCD0
:100D40009FE090FC9A12537F12540BFF90FCAA1262
:100D50005385F990FE38E02402FD1256291257639C
:100D6000FED39F4004AF06800D12570212543B126F
:100D7000538512540BFF90FCAA1253851255A48080
:100D80000D90FE38E02403125628F0020C6390FC0C
:100D9000A5125526404E12573A90FC9A12538512CE
:100DA0005403FD90FCAA1253851256DAED1219D99C
:100DB0001257A312538512540BFF90FCA5E0240197
:100DC00012556A1253851255A412570212543B123F
:100DD000538512540B1255631253851255A41257A2
:100DE0002112548E12579B020C5A125435125385FD
:100DF00012540B1255CC020C3A1255D790FC971294
:100E000053851253F340030211051253C854E06492
:100E1000806003020EAE1256AD90FC9A12538512FA
:100E20005495C39F40030211051254B46480706F3F
:100E30001255C190FC9712538512538D1255AD1265
:100E400053D312549C04F012564D1253851254037E
:100E50004FFF90FCAD125385F9EF12557E1253856A
:100E60001253BD1255AD1253D312549C1255161283
:100E700053851254034FFF90FCAD125385125585D4
:100E800090FC971253851253BD1255AD1253D312D5
:100E9000549C1255161253851254034F0210D81247
:100EA000543512538512540B1255CC020E1990FC76
:100EB000971253851253BD1253D012542A020DFCBF
:100EC0001255D790FC971253851253F3400302102A
:100ED000351253C8FF54E0642060030210231254FB
:100EE0004312568C1255F4D39F50D81256AD90FC35
:100EF0009A125385125495C39F400302101D125439
:100F0000B46420600302100E1255C112564390FCC7
:100F1000A1E012549CD39F50D590FC971253851298
:100F200053BD12554612564A125385125403547F2C
:100F30006F6003020FD790FCA5E0C3942D4003021D
:100F40000FD712573A125404FD90FCAA125385127F
:100F500056DAED1219D990FCA0E02481FDE433FCAF
:100F600090FC97125385125403FD1257A312538518
:100F700012540B5DFF90FCA5E0FE240112556A128D
:100F800053851255A48E82758300121978547864A3
:100F900001701612537812540B12570112551B127E
:100FA00053851254035FFF802212537812540B12A0
:100FB000570112551B125385125403FEC39F500450
:100FC000AF06800712537812540BFF125564125368
:100FD000851255A412572190FCA5E0FF602790FCD4
:100FE000971253851253BD125546547FFEEF24FDD0
:100FF000FDEC34FFFC90FCAA125385125403547F7D
:101000006E6005800012548E12579B020F0E125410
:101010003512538512540B1255CC020EEE1257871F
:10102000020EE490FC971253851253BD1253D01256
:10103000542A020EC31255D790FC971253851253AF
:10104000F340030211051253C854E06480600302A8
:1010500010F31256AD90FC9A125385125495C39F0B
:1010600040030211051254B4648070781255C19087
:10107000FC9712538512538D1255AD1253D312544F
:101080009C04F012564D1253851254035FFF90FCDE
:10109000AD125385F9EF12557E1253851253BD12CE
:1010A00055AD1253D312549C125516125385125437
:1010B000035FFF90FCAD12538512558590FC97128B
:1010C00053851253BD1255AD1253D312549C125571
:1010D000161253851254035FFF90FCAD1253851214
:1010E00056A5802112543512538512540B1255CC3B
:1010F00002105590FC971253851253BD1253D01213
:10110000542A0210381255D790FC97125385125367
:10111000F340030214631253C854E0646060030296
:10112000140F1256AD90FC9A125385125495C39F1A
:1011300040030214631254B464606003021400128A
:1011400055C190FC971253851253BD125545125646
:101150003AA3E004F012575C6003021263A3F0A309
:10116000F01255FE4008125658400302136D90FCD1
:10117000A6E0C3940C40030212581254DE64064EDB
:101180006018EF64084E6012EF64094E600CEF6463
:101190000A4E6006EF640B4E703790FC9712538531
:1011A0001253BD1253DA1254C4125385125403FE63
:1011B000EFD39E400F90FC971253851253BD1253EC
:1011C000DA02122712567212538512540BFF0212C2
:1011D000271254DE1256E5503790FC9DE030E12294
:1011E0001256EE12538512540BFF90FCB012538529
:1011F00090FCA61256DD1219786F600312548E020D
:10120000122790FC971253851253BD1253DA8017A0
:1012100090FC971253851253BD1253DA1254C41224
:1012200053851254034FFF90FCB0125385F990FC84
:10123000A61254A71254DE1256E5401C90FC9712D9
:1012400053851253BD125693FD90FCB01253851274
:10125000540B6D600312548E12550F7003125550CB
:10126000021161E412553E1255FE400302136D1245
:101270005658400302136D90FCA6E0C3940C400343
:101280000213621254DE64064E6018EF64084E606A
:1012900012EF64094E600CEF640A4E6006EF640BB7
:1012A0004E703790FC971253851253BD1253DA12C9
:1012B00054C4125385125403FEEFC39E500F90FC8A
:1012C000971253851253BD1253DA0213311256721C
:1012D00012538512540BFF0213311254DE1256E5DD
:1012E000503890FC9DE030E1231256EE12538512E7
:1012F000540BFF90FCB0125385F990FCA61256DEF9
:101300001219786F600312548E02133190FC9712F9
:1013100053851253BD1253DA801790FC97125385F0
:101320001253BD1253DA1254C41253851254035F80
:10133000FF90FCB0125385F990FCA61254A71254EA
:10134000DE1256E5401C90FC971253851253BD12D5
:101350005693FD90FCB012538512540B6D6003122E
:10136000548E12550F700312555002126790FCB044
:10137000125385F974031257C7125385F91255E5B4
:1013800090FC9DE030E20A90FCB0125385F91256B1
:10139000C012573250037405F090FCA6E0FFC394CE
:1013A00007402F90FCB01253852405F9E43AFA1255
:1013B000195F54BF1257C7125385F99000061219CE
:1013C00078FEC3942D500280027E2D900006EE120E
:1013D00019D990FCA0E0247FFDE433FC90FC971227
:1013E0005385125403541F6F600312548E90FCA255
:1013F000E00490FCA0F0A3E00490FC9FF0021463D2
:1014000012543512538512540B1255CC02112590EB
:10141000FC971253851253BD1253D012542A021155
:101420000890FC9712538512563054FD12557E12C7
:10143000538512572912548E90FC9A1253851254D8
:10144000E7125385F912AE4612546290FCAA125369
:1014500085121853125385F912B42F90FE36E0709E
:1014600002D22F90FC971253851255DE640160035F
:101470000217D390FCA4E0C39401500A1254F61250
:101480005385F912AE4690FE36E0B4042A90FD2250
:101490007401F0A374FCF0A374A5F090FCADE0F926
:1014A000A3E0FAA3E090FD2512547D90FCAA12530C
:1014B00085F912A91C801690FCA5E0C39403500D79
:1014C00012546290FCAA125385F912AC6F12573273
:1014D000501890FDB97401F0A374FCF0A374A6F049
:1014E00090FCB0125385F912B42FD3125733400336
:1014F0007405F0E412553E125413501690FCA712D6
:10150000538512540320E70A12550F70EA12555002
:1015100080E5125523400F90FCA7125385F912194C
:101520005F44801219C7E490FCA0F090FC9712531E
:10153000851253BD1255ADF9EE3AFA740212557E7A
:101540001253851253BDFF04F0E92FF9EE3AFA74F5
:10155000031219C790FCA4E0240BFFA3E02FFFA304
:10156000E02FFF90FC971253851253BD12545790F1
:10157000FCA5E075F01E841219A512568C90FCA3F0
:10158000E0FF90FC971253851253BDFE04F0EE125B
:10159000545990FCA4E04440FF90FC9712538512EC
:1015A00053BDFE04F0EE125459E412553E1254138A
:1015B000502090FCA7125385125403FF90FC971201
:1015C00053851253BD12545312550F70E0125550EB
:1015D00080DB90FCA5E0C3941E500302165D90FCD6
:1015E000971253851253BD1255ADF9EE3AFA743E77
:1015F0001219C7E412553E1254DEC3941EEE6480E5
:101600009480502090FCAA12538512540BFF90FC3A
:10161000971253851253BD12545312550F70D8129E
:10162000555080D390FCA5E024E2FFE434FFFE9007
:10163000FCAA125385241EF9E43AFAC003C00290B2
:10164000FCAAA3E0FAA3E0F8AC02AD03D002D003F9
:1016500012193990FCA5E024E2F00215D290FCA505
:10166000E04420FF90FC971253851253BD1254534F
:10167000E412553E90FCA5125416502090FCAA127C
:101680005385125403FF90FC971253851253BD12D9
:10169000545312550F70DD12555080D890FC97129C
:1016A00053851253BD1255ADF9EE3AFA74831219EF
:1016B000C790FCAD125385F912195FFF90FC971289
:1016C00053851253BD12545390FCAD125385F990BB
:1016D00000011255B91253851253BDFE04F0EE12EB
:1016E000545990FCAD1253851255B51253851253BF
:1016F000BDFE04F0EE12545990FCA6E04460FF9049
:10170000FC971253851253BDFE04F0EE125459E4B7
:1017100012553E90FCA6125416502090FCB0125365
:1017200085125403FF90FC971253851253BD125437
:101730005312550F70DD12555080D8E412553E12E9
:101740005413506290FCA0E0C3946E505990FCA7D3
:10175000125385125403547FFF6401603EEFC3941B
:101760003C5038EF75F012A42481F9744835F0FA32
:101770007BFFC003C002C00190FC97125385125337
:10178000BD7E0029F9EE1256D3D001D002D0037FDE
:101790001212193990FCA0E02412F012550F7003B8
:1017A00012555002173F90FCA0E0FFFDC374809DCE
:1017B000FDE49400FCC004C00590FC971253851210
:1017C0005755EF7C0029F9EC3AFA7D00D007D00696
:1017D00012227B1255391254DEC3947FEE6480943A
:1017E00080501390FC9712538512540B12550870B9
:1017F000E512555080E01257AE125385F990007FE4
:10180000EF1219D91255DF6401704290FC97125300
:1018100085F99000FEE41219D91255391254DEC32D
:10182000947FEE64809480501690FC97125385123A
:1018300057551253E812550970E212555080DD12C7
:1018400057AE125385F99000FFEF1219D990FC9E04
:10185000E0FF22F912AC6F90FDB97401F0A374FCA3
:09186000F0A374A6F090FCB02284
:102E5D0049646C65005472616E736D69745F4D6584
:102E6D007373616765005365745F4C6F6769636168
:102E7D006C5F4164647265737300436F6E6E65635E
:102E8D007400446973636F6E6E656374005374618F
:102E9D006E646279005374616E6462795F416C6C2B
:102EAD00005265636F72645F43757272656E740074
:102EBD005265636F72645F43757272656E745F4FB6
:102ECD006666005365745F54696D65725F50726F0D
:102EDD006772616D00436C6561725F54696D6572F7
:102EED005F50726F6772616D004765745F4D656EFF
:102EFD00755F4C616E677561676500416E6E6F75CC
:102F0D006E63655F4D656E755F4C616E677561676C
:102F1D006500436F6E74726F6C5F4465636B005335
:102F2D00656C6563745F54756E65725F536572761B
:102F3D0069636500436F6E74726F6C5F54756E6577
:102F4D00720053656E645F56656E646F725F436F9A
:102F5D006D6D616E640042726F6164636173745F65
:102F6D0056656E646F725F436F6D6D616E64005672
:102F7D00656E646F725F52656D6F74655F427574D7
:102F8D00746F6E5F507265737365640056656E6421
:102F9D006F725F52656D6F74655F427574746F6E9D
:102FAD005F52656C6561736564005265717565731B
:102FBD00745F4D656E7500557365725F436F6E740A
:102FCD00726F6C5F507265737365640055736572D3
:102FDD005F436F6E74726F6C5F52656C6561736584
:102FED006400526571756573745F53797374656DA3
:102FFD005F417564696F5F4D6F6465005570646105
:10300D0074655F4465766963655F496E666F0052EE
:10301D006571756573745F496D6167655F56696547
:10302D00775F4F6E00526571756573745F54657887
:10303D00745F566965775F4F6E00416E6E6F756E8A
:10304D0063655F4163746976655F536F7572636520
:10305D00005365745F496E6163746976655F536F84
:10306D007572636500526571756573745F4469733C
:10307D00706C61795F4F53445F537472696E670072
:10308D00496E666F726D5F4D656E755F53746174D9
:10309D007573005365745F53797374656D5F417516
:1030AD0064696F5F4D6F6465005265706F72745F18
:1030BD005265636F72645F5374617475730052650A
:1030CD00706F72745F54696D65725F53746174755E
:1030DD0073005265706F72745F54696D65725F43F2
:1030ED006C65617265645F53746174757300556EC0
:1030FD00737570706F727465645F4D65737361671E
:10310D006500496D6167655F566965775F4F6E0054
:10311D00546578745F566965775F4F6E00416374CF
:10312D006976655F536F7572636500496E6163748F
:10313D006976655F536F757263650052657175656C
:10314D00737465645F666F725F5374616E646279E8
:10315D0000496E666F726D65645F4D656E755F4C8F
:10316D00616E677561676500526563656976656453
:10317D005F56656E646F725F436F6D6D616E640057
:10318D0052656365697665645F56656E646F725FDF
:10319D0052656D6F74655F427574746F6E5F5072BA
:1031AD0065737365640052656365697665645F5622
:1031BD00656E646F725F52656D6F74655F42757495
:1031CD00746F6E5F52656C656173656400446973FD
:1031DD00706C61795F4F53445F537472696E670011
:1031ED00496E666F726D65645F4D656E755F537484
:1031FD00617475730052656365697665645F5573B7
:10320D0065725F436F6E74726F6C5F50726573732E
:10321D0065640052656365697665645F55736572B3
:10322D005F436F6E74726F6C5F52656C6561736531
:10323D00640053797374656D5F417564696F5F4D9B
:10324D006F64655F536574004465766963655F49B6
:10325D006E666F5F4368616E676564005365745F8A
:10326D0053747265616D5F5061746800526571755C
:10327D0065737465645F5265636F72645F437572E5
:10328D0072656E74005265717565737465645F5215
:10329D0065636F72645F43757272656E745F4F66BE
:1032AD0066005265717565737465645F5365745F0F
:1032BD0054696D65725F50726F6772616D00526512
:1032CD00717565737465645F5365745F54696D657D
:1032DD00725F50726F6772616D5F5469746C6500D7
:1032ED005265717565737465645F436C6561725F7A
:1032FD0054696D65725F50726F6772616D005265D2
:10330D00717565737465645F666F725F4D656E751B
:10331D00005265717565737465645F436F6E747289
:10332D006F6C5F4465636B0053656C6563746564B6
:10333D005F54756E65725F53657276696365005291
:10334D0065717565737465645F436F6E74726F6CD0
:10335D005F54756E65720052657175657374656441
:10336D005F666F725F53797374656D5F41756469E4
:10337D006F5F4D6F646500526F7574696E675F4F57
:10338D00666600443D307825302E32582044656500
:10339D007020436F6C6F722044657465637465644F
:1033AD000D0A00443D307825302E32582034204F00
:1033BD00757470757420537570706F72740D0A008A
:1033CD00443D307825302E325820547820545245C3
:1033DD0047203D20307825302E32580D0A004552B9
:1033ED00524F523A204E3D307825302E32582041E2
:1033FD004B535620524459202D204D4355204949B9
:10340D00432025640D0A004552524F523A204E3D3D
:10341D00307825302E325820414B5356207265613D
:10342D0064202D204D4355204949432025640D0A24
:10343D00004552524F523A204E3D307825302E32B3
:10344D005820414B53562072656164202D204B65E9
:10345D00792057726F6E670D0A004552524F523ADE
:10346D00204E3D307825302E325820547820526928
:10347D002072656164202D204D435520494943201C
:10348D0025640D0A004552524F523A204E3D307878
:10349D0025302E325820424B5356207265616420E0
:1034AD002D20444E204444432025640D0A004552EE
:1034BD00524F523A204E3D307825302E3258204210
:1034CD004B53562072656164202D204B6579205732
:1034DD00726F6E670D0A004552524F523A204E3DA3
:1034ED00307825302E32582052782052692072655E
:1034FD006164202D20444E204444432025640D0A50
:10350D00004552524F523A204E3D307825302E32E2
:10351D0058204B5356204649464F20726561642012
:10352D002D20444E204444432025640D0A0045526D
:10353D00524F523A204E3D307825302E3258204B86
:10354D005356204649464F2072656164202D204B0D
:10355D0065792057726F6E670D0A004552524F52B2
:10356D003A204E3D307825302E325820454449447E
:10357D002062302072656164202D20444E20444429
:10358D00432025640D0A004552524F523A204E3DBC
:10359D00307825302E325820454449442043686503
:1035AD00636B206661696C65642C207045444944E9
:1035BD005B3132365D3D307825302E3258203E203D
:1035CD00380D0A004552524F523A204E3D30782563
:1035DD00302E32582045444944206269207265617D
:1035ED0064202D20444E204444432025640D0A00C0
:1035FD004552524F523A204E3D307825302E32589A
:10360D00204544494420636865636B73756D20657F
:10361D0072726F720D0A005741524E494E473A2051
:10362D00443D307825302E3258204E6F2045504382
:10363D00432064657465637465640A0D00443D3010
:10364D007825302E325820455043432064657465EB
:10365D0063746564205665723D25642E25640A0DDC
:10366D00005741524E494E473A204E6F20446576E1
:10367D0069636520666F756E640D0A005741524E81
:10368D00494E473A204E6F20417564696F2053793A
:10369D007374656D20666F756E640D0A0057415227
:1036AD004E494E473A20443D307825302E32582031
:1036BD0045504343204576656E74204D697373699B
:1036CD006E670D0A004552524F523A20443D3078F4
:1036DD0025302E3258204550434320436F6D6D6188
:1036ED006E642054696D652D6F75740D0A00455219
:1036FD00524F523A20494943206661696C656420F6
:10370D0025642C20494943416464723D307825304D
:10371D002E32582C20526567416464723D307825F5
:10372D00302E32580D0A00FF2E5DFF2E62FF2E73D4
:10373D00FF2E87FF2E8FFF2E9AFF2EA2FF2EAEFF9C
:10374D002EBDFF2ED0FF2EE2FF2EF6FF2F08FF2FEE
:10375D001FFF2F2CFF2F41FF2F4FFF2F63FF2F7CBC
:10376D00FF2F99FF2FB7FF2FC4FF2FD9FF2FEFFF8B
:10377D003009FF301CFF3032FF3047FF305EFF3025
:10378D0072FF308DFF30A0FF30B6FF30CBFF30DF42
:10379D00FF30FBFF310FFF311DFF312AFF3138FFA5
:1037AD003148FF315EFF3175FF318DFF31B3FF3190
:1037BD00DAFF31EDFF3202FF3220FF323FFF32558B
:1037CD00FF3269FF3279FF3292FF32AFFF32CBFF0A
:1037DD0032EDFF330BFF331EFF3335FF334CFF3319
:0437ED0064FF3384BE
:0C8E6D0001680042FCD900000264000013
:106F3C0090FD28E0FBA3E0FAA3E0F912195FFF90A3
:106F4C00FD2BE0FBA3E0FAA3E022F090FCDFE4755C
:106F5C00F001121AAEFE748025F0F58274FF3EF536
:106F6C00837469F090FCDFE475F001121AAEFE74C4
:106F7C008025F0F58274FF3EF58322F912195F0427
:106F8C00FF90FD9A7B00E47A007922F0A304F022B2
:106F9C00F0A3EDF0A3EBF0A3EAF0A3E9F0221219B1
:106FAC005F04FF90FD597B00E47A007922F0A32264
:106FBC00F912195FFF90FBCAE4F0A3EFF02290FFE7
:106FCC0080F090FCEBE47B017AFF7980F0A322F94E
:106FDC009000010219782407F9E43AFA90FD59E47B
:106FEC00F0A322F912195FFF90FE1FE4F0A3042214
:106FFC007B007A00792290FCEBE4F0A322F91219C1
:10700C005FFFE490FE1FF0A32290FCDBE090FBCC32
:10701C00FFE4F0A3EFF022F990FCDFE0FEA3E0F533
:10702C00828E83021978F9900002121978FF900071
:10703C0003121978FD22F912195FFF7B017AFF798F
:10704C0080227967E7C4F8540FC868FF19E7C45465
:10705C00F048FEE42FFDEE22F9A3E0FFA3E090FC44
:10706C00EBCFF0A3EFF0222FF9EA3EFA90000412D6
:10707C001978FF900005121978FD2290FCDBEFF0D7
:10708C00E0FE2204F0A3F07D74FF22F990FD9AE457
:10709C00F0A3222401F9E43AFA02195FE490FCDF30
:1070AC00F0A3F0227405F0E4A3F07D757F0122F9C2
:1070BC0012195F04FF2290FD43E0FD90FBCAE4F03F
:1070CC00A3EDF0A32290FCDFE0FDA3E090FD59CDF1
:1070DC00F0A3EDF022A3E4F0A3E522F07BFF7A33DA
:1070EC0079CD2290FCDFE4F0740AA3F0E4A3F0A3C2
:1070FC00F02290FCE0E004F02290FCDFE004F022AF
:10710C0090FDD9E014FF90FDD8E02290FCDFE0FE6A
:10711C00A3E0FFC39406EE6480948022D390FCE03D
:10712C00E0940090FCDFE064802290FCE2E004F04C
:10713C002290FCE1E004F022C390FCE2E094039086
:10714C00FCE1E064809480227480F0E4A3F07DA1E3
:10715C007F012290FCDBE0FF90FBCC22E025E0FFDE
:10716C0090FCDFE033FE90FCE322C390FE5CE094E5
:10717C00E890FE5BE0940322A3E024FDF090FCDF9A
:10718C00E034FFF02204F0A3F07DA0FF2290FE1E5D
:10719C00E0FF7401A8070822E52225E0F52222F081
:0971AC00A37402F07D747F01223E
:108A5F0090FCDC126FA190FDBFE0F9A3E0FAA3E058
:108A6F0090FCE3C9126FA290FCE3126F4E127032AA
:108A7F0012795190FCE3126F4E1270327B02126921
:108A8F00A790FCE3126F4EF912195FFF126FDCFD16
:108A9F00127AB890FCE3126F4EF912195FFF126F42
:108AAF00DCFD7B011269A712AE767D087F06127975
:108ABF00517B017D087F061269A71270A8127117EA
:108ACF00501FEF25E0FFEE33FE90FCE3126F4E12C6
:108ADF0070737B011269A71270FE7003127105800B
:108AEF00DCE4FB7D01FF12ACDB7B02E4FD7F0112B6
:108AFF00ACDB7BFF7AA2795FE4FF12B54C90FE608E
:108B0F0074FEF07BA0E4FD12AB157BFF7A00794E6B
:0A8B1F00E4FF12B53B7D0102AA1F1E
:10AE760090FCE3126F4EF912195FFF126FDCFD12A0
:10AE86007AB812985990FCE3126F4EF912195FFFC7
:0CAE9600126FDCFD1279517F0402B5CD73
:10B4F00090FCE3126F4E1270321279517D02E4FF1C
:03B5000002B1B2E3
:10B52900E4FDFF12B1B290FCE3126F4E12703202C9
:02B539007AB8DE
:1095EA0090FE76126FA190FE76126F4EF9ED121967
:1095FA00C790FE76126F4EF9900001E41219D91243
:10960A006F887D05128B2990FCDBE07024E52260CF
:10961A002090FE76126F4E126FBC7BFF7A337990E0
:10962A0012A71E90FE76126F4E12709F44401219B6
:10963A00C775220890FE76126F4EF912195F126FE3
:10964A008C7D07128B2990FE76126F4E126F877DE2
:10965A0007128B2990FCDBE0702330132090FE76F2
:10966A00126F4E126FBC7BFF7A3379B012A71E902D
:0E967A00FE76126F4E12709F44801219C722A6
:0DB5A700126FDC30E6047F0180027F00227D
:109AA50090FE79126FA190FE79126F4E126FDB3026
:109AB500E51F30E60820E74C126FF0802690FE790E
:109AC500126F4E126FEF129B26126F4E126FEF80C0
:109AD5002B90FE79126F4E126FDB30E60D20E724D6
:109AE50012700AF07B067D06801790FE79126F4E84
:109AF500127009129B26126F4E127009F07B047DBD
:109B05000A12A89390FE79126F4E126F877D061286
:109B15008B2990FE79126F4E126FBC1270E102A76D
:0D9B25001EF07B057D0A12A89390FE7922A8
:10AF260090FE7C126FA1ED90FE7C600A126F4E12AD
:10AF3600709F44208008126F4E12709F54DF1219C2
:0BAF4600C790FE7C126F4EF9029AA526
:10A6830090FE7F126FA190FE7F126F4E126FDB3030
:10A69300E40830E61C12700A800F90FE7F126F4EA2
:10A6A300126FDB30E60B126FF0F07B077D0612A80A
:10A6B3009390FE7F126F4E126F877D06128B299047
:0EA6C300FE7F126F4E126FBC1270E102A71ED6
:10AF510090FE82126FA1ED90FE82600A126F4E1276
:10AF6100709F44108008126F4E12709F54EF121997
:0BAF7100C790FE82126F4EF902A6830B
:10AB8D0090FE85126FA190FE85126F4E126FDB3015
:10AB9D00E60B126FF0F07B057D0612A89390FE85F3
:10ABAD00126F4E126F877D06128B2990FE85126FE4
:0AABBD004E126FBC1270E102A71ED9
:10AEA20090FE88126FA190FE88126F4E126FDB30F7
:10AEB200E70812700AF07B03800C90FE88126F4E36
:0CAEC200127009F07B017D0712A893229A
:109E580090FE8B126FA190FE8B126F4E126FDB304B
:109E6800E63475220812195F126F8C7D05128B2952
:109E780090FE8B126F4E126FDB30E7057522C280A1
:109E88000A75229690FE8B126F4EF912195F126FA7
:109E98008C7D06128B2990FE8B126F4EF9129AA5B3
:109EA80090FE8B126F4EF912A68390FE8B126F4EA6
:109EB800126FDB30E708126FF0F07B03800B90FE27
:0F9EC8008B126F4E126FEFF0FB7D0712A89322E3
:10ADE30090FE8E126FA190FE8E126F4E126F877DB2
:10ADF30007128B2990FE8E126F4E126FDB30E7081D
:10AE0300A216821782138006A21682178211E433D8
:02AE1300FF221C
:0EB57D00126F887D07128B29A215E433FF227E
:10B44600126F887D07128B2990FCDBE060037F0179
:07B4560022A214E433FF22DF
:0EB58B00126F887D08128B29A216E433FF226E
:0EB59900126F887D40128B29A210E433FF222E
:10000E0012195FFF90FDC5126F4E1270977403F0B8
:05001E007D50028B295A
:10B3CF0012195FFF90FD6E126F4EF9A3E0FD127020
:08B3DF0098EDF07D80028B293E
:10B4740012195F04FF90FDCB126F4E12709774087F
:06B48400F07D41028B295E
:1000560012195FFF90FDD1126F4E1270977414F053
:050066007D60028B2902
:10B2E00090FE91126FA190FE91126F4EF912A497E9
:10B2F00090FE91126F4E127009F0FB7D0802A89328
:10B1F90090FE94126FA190FE94126F4EF912A497CB
:10B2090090FE94126F4E126FEFF0E4FB7D0802A8D6
:01B2190093A1
:10B21A0090FE97126FA190FE97126F4EF912A497A3
:10B22A0090FE97126F4E126FEFF07B077D0802A80F
:01B23A009380
:10B23B0090FE9A126FA190FE9A126F4EF912A4977C
:10B24B0090FE9A126F4E127009F07B077D0802A8D0
:01B25B00935F
:10B25C0090FE9D126FA190FE9D126F4EF912A49755
:10B26C0090FE9D126F4E126FEFF0E4FB7D0F02A863
:01B27C00933E
:10B3000090FEA0126FA190FEA0126F4EF912A497AA
:10B3100090FEA0126F4E127009F0FB7D0F02A893F1
:10A0BD0090FE39126FA1A3EDF012A49790FE391204
:10A0CD006F4E126F877D09128B293011037F01228C
:10A0DD0090FE3CE0FF12A53FE4F522FB90FCEB1255
:10A0ED006F93A3F07D60FF1277A6E4F522FB90FC41
:10A0FD00EB126FB51271911277A6127087C0069090
:10A10D00FCEB126F901271571277A6D0E04F90FCB6
:0AA11D00DBF070037F02227F0022B6
:1000260090FEA3126FA190FEA3126F4EF912A49731
:1000360090FEA3126F4E126F877D09128B29A212B2
:04004600E433FF227E
:10B27D0090FEA6126FA190FEA6126F4EF912A49722
:10B28D0090FEA6126F4E126FEFF0E4FB7D0E02A83A
:01B29D00931D
:10B3200090FEA9126FA190FEA9126F4EF912A49778
:10B3300090FEA9126F4E127009F0FB7D0E02A893C9
:10B29E0090FEAC126FA190FEAC126F4EF912A497F5
:10B2AE0090FEAC126F4E126FEFF07B047D0F02A872
:01B2BE0093FC
:10B2BF0090FEAF126FA190FEAF126F4EF912A497CE
:10B2CF0090FEAF126F4E127009F07B047D0F02A833
:01B2DF0093DB
:10AECE0090FD72126FA190FD72126F4EF912A4973F
:10AEDE0090FD72126F4EF912195FFF90FD76126F90
:0CAEEE004E1270977408F07D15028B293D
:10AA9B0090FE3D126FA1A3EDF012A49790FE3D1214
:10AAAB006F4E126F877D0F128B2990FCDBEFF060DE
:10AABB00167BFF7A3379EB90FE40E0126FC0127079
:0DAACB001512A71E7F0022A217E433FF2200
:1093630090FD79126FA1A3EDF012A49790FD7912ED
:109373006F4E1270BB90FD7D126F4E127097740783
:10938300F07D1D128B2990FCDBEFF060127BFF7ADE
:1093930034791490FD7CE0126FC012715F80581213
:1093A30070A8A3F0A3F0F522752201E522601A90BC
:1093B300FD7D126F4E1270235522600812713670B4
:1093C3000312713D1271A480E21270FE70031271D8
:1093D3000590FCDFE07004A3E0640570CB90FCE132
:1093E300E07004A3E0641460197BFF7A34793E9043
:1093F300FD7CE0FF90FBCAE4F0A3EFF012A71E7F11
:0594030000227F0122A0
:10AEFA0090FD80126FA190FD80126F4EF912A497F7
:10AF0A0090FD80126F4EF912195FFF90FD84126F47
:0CAF1A004E1270977405F07D10028B2918
:10AFA70090FEB2126FA190FEB2126F4EF912A497E3
:10AFB70090FEB2126F4E126F877D0F128B29E5221A
:0AAFC70030E1047F0180027F0022C8
:10A84D0090FD87126FA1A3EDF012A49790FD8712D2
:10A85D006F4E1270BB90FD8B126F4E12709774027B
:10A86D00F07D22128B2990FCDBEFF060167BFF7AD6
:10A87D0034796790FD8AE0126FC012701512A71E11
:06A88D007F00227F012282
:10AFD10090FD8E126FA190FD8E126F4EF912A49703
:10AFE10090FD8E126F4E1270BB90FD92126F4E1239
:0AAFF10070977408F07D25028B298B
:1091500090FE42126FA190FE41EFF012A53F90FEEB
:1091600042126F4EF9E41219C790FE42126F4EF987
:1091700012700212708F1277A6127087C00690FECE
:1091800042126F4EF91270021270B01277A6D0E040
:109190004F90FCDBF060127BFF7A34799290FE41B5
:1091A000E0126FC012715F80561270A8A3F0A3F096
:1091B000752201E522601A90FE42126F4E12702352
:1091C00055226008127136700312713D1271A4802D
:1091D000E21270FE700312710590FCDFE07004A3D0
:1091E000E0640570CB90FCE1E07004A3E0641460DF
:1091F000197BFF7A3479BB90FE41E0FF90FBCAE413
:0D920000F0A3EFF012A71E7F00227F0122D5
:10B3400012A53F75224090FCEB126FB212708F1263
:0FB3500077A6126FFC041270B21277A6AF2222FA
:10B0780090FEF2EDF012A53F752215126FFC1270CA
:10B088008F1277A67B017AFE79F212700204F0A380
:09B0980004F07D747F010277A62B
:1001D90090FEB5126FA112A53F752218126FFC127D
:1001E900708F1277A690FEB5126F4EF912700274D5
:0701F900081271AB0277A6AA
:10B0CA0090FEB8126FA112A53F752210126FFC12E2
:10B0DA00708F1277A690FEB8126F4EF91270027432
:07B0EA00051271AB0277A60D
:10A2C50090FE46126FA190FE45EFF012A53F90FE5D
:10A2D50046126F4EF974081219C790FE46126F4E5A
:10A2E500F912700212708F1277A6127087C006904D
:10A2F500FE46126F4EF912700274021270B2127796
:10A30500A6D0E04F90FCDBF060167BFF7A3479E451
:10A3150090FE45E0126FC012701512A71E7F002235
:03A325007F012293
:10AC010090FEBB126FA112A53F90FEBB126F4EF9D1
:10AC110074411219C790FEBB126F4EF912700212E5
:10AC2100708F1277A690FEBB126F4EF912700274EC
:07AC3100021270B20277A6C7
:10AC380090FEBE126FA112A53F90FEBE126F4EF994
:10AC480074201219C790FEBE126F4EF912700212CC
:10AC5800708F1277A690FEBE126F4EF912700274B2
:07AC6800141270B20277A67E
:1082620090FDD5126FA190FDD4EFF012A53F90FDC5
:10827200D8E0703B752243FB7A00792290FCEBF048
:10828200A312708F1277A612710C90FDD5B5070C50
:10829200126F4EF91270021270B0803D126F4EF9D9
:1082A2001270027405F0A37401F07D75FF802A122A
:1082B200710C90FDD5B5070F126F4EF91270027452
:1082C20005F0A37402800D126F4EF912700274054C
:1082D200F0A37403F07D757F011277A690FCDBEFAB
:1082E200F090FCDBE0FF60177BFF7A35790E90FDA2
:1082F200D41270C5E4F0A3EFF012A71E7F00221281
:1083020070A8A3F0A3F0752201E522601A90FDD5B2
:10831200126F4E12702355226008127136700312CA
:10832200713D1271A480E21270FE70031271059009
:10833200FCDFE07004A3E0640570CB90FCE1E07028
:1083420004A3E0641460327BFF7A35793B90FDD45C
:10835200E0126FC012A71E12710C6F601990FDD54A
:10836200126F4EF9E490FCEBF0A3F0A37402F07DDF
:0C837200757F011277A67F00227F012298
:1073EA0090FD44126FA190FD43EFF012A53FE49087
:1073FA00FF80F090FCEB126FD21275DEE490FF80F2
:10740A00F012704790FCEBF0A31271911277A6125A
:10741A007087C00690FD44126F4EF9127002127105
:10742A00541277A6D0E04F90FCDBF060137BFF7A12
:10743A0035796890FD43E0126FC012715F027520C2
:10744A0090FD44126F4EF990007E121978FFD39482
:10745A000840141270C2E4F0A3EFF07BFF7A35798A
:10746A009412A71E7F052290FD44126F4EF99000D8
:10747A007E12197890FD48F090007EE41219D9E442
:10748A0090FD49F090FD4704F090FD48E0FF90FD23
:10749A0047E0FED39F4003027537EEC313126FCA4B
:1074AA001275DE90FD47E05401C433333354801221
:1074BA006FCA1271911277A6127087C006126FCE28
:1074CA001271541277A6D0E04F90FCDBF090FF8047
:1074DA00E06402703190FD49E0702B04F090FD44A5
:1074EA00126F4E2480F9E43AA801FCAD03127047EA
:1074FA007E007F8012193990FD44126F4EF9900078
:10750A007E74011219D990FCDBE0FF60177BFF7AC9
:10751A003579D11270C2E4F0A3EFF012A71E90FCE5
:10752A00DBE0FF2290FD47E004F002749390FD44F3
:10753A00126F4EF9E41219C790FD44126F4EF9907A
:10754A00000174FF1219D990000274FF1219D99020
:10755A00000374FF1219D990000474FF1219D9900C
:10756A00000574FF1219D990000674FF1219D990F8
:10757A000007E41219D9E490FD4AF01270A990FDAF
:10758A0049E060067E017F0080047E007F80C39010
:10759A00FCE0E09FEE6480F812712F98501A90FD7B
:1075AA0044126F4E127023FF90FD4AE02FF01270C2
:1075BA00FE70CB12710580C690FD4AE060137BFF16
:1075CA007A3579FD90FD43E0126FC012A71E7F063F
:0F75DA00227F002204F0A3F07D60FF1277A6222B
:109FCE0090FEC1126FA1ED1219C790FEC1126F4E15
:109FDE001270BB90FD59126FD17402F07D007C049B
:109FEE001288C190FCDBEFF090FEC1601C126F4E28
:109FFE00126FBC7BFF7A36792412A71E90FEC11217
:10A00E006F4EF9900001E4802B126F4E126FBC90D0
:10A01E00FF8012701890FF81E090FBCE12701C7BB7
:10A02E00FF7A36794A12A71E90FEC1126F4EF99032
:08A03E00000174011219D9227E
:10846E0090FE49126FA1A3EDF090FE49126F4E4A95
:10847E004B700302855590FE49126F4E126FDB2032
:10848E00E0030285551270A890FCDF126F7474120F
:10849E00126F6F74DE126F6F740FF01270431270E2
:1084AE00D17D027C011288C11270A890FE4CE0FFB3
:1084BE0090FCDFE475F001121AAEFC748025F0F525
:1084CE008274FF3CF583EF126F6F74FF126F6FE4CF
:1084DE00F090FCDF126F747463126F6F7468126F1A
:1084EE00567445126F6F7458126F6F7450126F6F0F
:1084FE007445126F6F7450126F6F742D126F6F740C
:10850E0053126F6F7470126F6F746C126F567474A7
:10851E00126F6F7474126F6F7465126F6F747212C4
:10852E006F6FE4F090FCDF126F74E4F090FCDF12DA
:10853E006F74E4F090FE49126F4E1270421270D1B9
:08854E007D097C011288C122A5
:10A4420090FE4D126FA1A3EDF090FE4D126F4E4A99
:10A452004B604190FE4D126F4E126FDB30E03512B1
:10A46200195FFF7D0412A38A90FE50E0F52290FE50
:10A472004D126F4EF912195F126FAE04F07D007C1F
:10A48200051288C190FE4D126F4EF912195FFF7DC1
:05A492000312A38A2261
:10AD110090FDDA126FA190FDDA126F4E4A4B60245A
:10AD210090FDDA126F4E126FDB30E01812195FFFDF
:10AD310090FDDD126F4EF9126FE87402F07D077C11
:05AD4100011288C1228F
:107EDD0090FD28126FA190FD28126F4E4A4B700332
:107EED00027FFF90FD28126F4E126FDB20E0030220
:107EFD007FFF126F4BF912195F24FE6074146071CD
:107F0D0014600D147003027FE024046003027FFFF0
:107F1D0090FD2E126F4EF912195F601DEA494B60EC
:107F2D001890FD28126F4EF912195FFF90FD2E1259
:107F3D006F4EF9126FE8128000126F3CF9126FE864
:107F4D0004F07D09FC1288C1126F3C2403126FE40A
:107F5D0012800B126F3C2406126FE404F07D0BFCB3
:107F6D001288C1126F3C126FE204F07D28FC027F73
:107F7D00FC90FD2E126F4EF912195F601DEA494BF0
:107F8D00601890FD28126F4EF912195FFF90FD2EAB
:107F9D00126F4EF9126FE8128000126F3CF9126FDA
:107FAD00E804F07D09FC1288C1126F3C2403126FA6
:107FBD00E412800B126F3C2406126FE404F07D0B6B
:107FCD00FC1288C1126F3C126FE27408F07D297C9F
:107FDD0001801C126F3CF9126FE804F07D0AFC124F
:107FED0088C1126F3C126FE27402F07D317C011278
:107FFD0088C122740EF07D127C011288C122740397
:09800D00F07D0F7C011288C122F4
:10AD460090FDE0126FA190FDE0126F4E4A4B602419
:10AD560090FDE0126F4E126FDB30E01812195FFFA4
:10AD660090FDE3126F4EF9126FE87403F07D0C7CD0
:05AD7600011288C1225A
:10A9E00090FD4B126FA190FD4B126F4E4A4B7003BE
:10A9F0007F012290FD4B126F4E126FDB20E0037F30
:10AA0000012212195F04FF90FD4E126F4EF9A3123E
:0FAA100070D47D007C071288C190FCDBEFF02230
:108BF30090FD31126FA190FD31126F4E4A4B7002FE
:108C0300FF2290FD31126F4E126FDB20E0037F00D5
:108C130022786676000876017866E6FE08E6FFC3EA
:108C2300940FEE94004003028CB0EF64054E606F26
:108C330090FD31126F4E1270BBC00712704E34029A
:108C4300FC126FAF04F0D0071288C1E522F4604F25
:108C5300E522604B90FD31126F4E1270BBC00712BC
:108C6300704E3402FC90FD34126F4EF9126FE874AB
:108C73000FF0D0071288C190FD31126F4E1270BBF6
:108C8300C00712704E3403FC90FD37126F4EF91279
:108C93006FE8740EF0D0071288C17867E6FF227878
:108CA3006706E6186003028C1B06028C1B7BFF7AA7
:098CB30036796E12A71E7F0F2214
:10A3280090FDE6126FA190FDE6126F4E4A4B700247
:10A33800FF2290FDE6126F4E126FDB20E0037F00D4
:10A3480022126FAA04F07D507C021288C1E522F423
:10A358006024E522602090FDE6126F4E1270BB90DB
:10A36800FDE9126F4EF9126FE87409F07D507C0216
:10A378001288C17F05227BFF7A36798912A71E7F52
:02A388000022B1
:10ACA50090FDEC126FA190FDEC126F4E4A4B6025A2
:10ACB50090FDEC126F4E126FDB30E01912195F0434
:10ACC500FF90FDEF126F4EF9126FE8740FF07D00E3
:06ACD5007C021288C1227E
:109F550090FE51126FA1A3EDF090FE51126F4E4A83
:109F65004B605A90FE51126F4E126FDB30E04EE49B
:109F750090FF80F0127043126FE804F0FDFC128828
:109F8500C190FF8074FF1270F790FE51126F4E1250
:109F95007042126FE8129FC37F0112B5D990FF80FE
:109FA5007405F090FE54E090FF81F0E4A3F090FE7C
:109FB50051126F4E127042126FE8129FC322740342
:099FC500F07D207C011288C1220C
:10AD7B0090FDF2126FA190FDF2126F4E4A4B6024C0
:10AD8B0090FDF2126F4E126FDB30E01812195FFF5D
:10AD9B0090FDF5126F4EF9126FE87408F07D207C70
:05ADAB00011288C12225
:10A1270090FD3A126FA1A3EDF090FD3A126F4E4ADF
:10A137004B605690FD3A126F4E126FDB30E04A12B9
:10A14700195FFF7B017AFD793D126FE804F0FDFC92
:10A157001288C190FD3A126F4EF912195FFF90FDF8
:10A1670040126F4EF990FD3FE0FD126FE8EDF07D74
:10A17700007C051288C190FD3A126F4EF912195FE3
:0AA18700FF90FD3EE0FD12A38A22C6
:109C460090FEC4126FA190FEC4126F4E4A4B700272
:109C5600C32290FEC4126F4E126FDB20E002C322B5
:109C6600D390FCDAE0942090FCD9E06480948040A4
:109C76001C90FEC4126F4E126FBC7BFF7A3679AA17
:109C860012A71EE490FCD9F0A3F07868F67868E68F
:109C9600603290FEC4126F4EF9126FAA04F07D0571
:109CA600FC1288C130110F7868E6600116E490FC5A
:109CB600D9F0A3F0D32290FCDAE004F0700690FC11
:069CC600D9E004F0C32206
:10A53F0090FEF3EFF01270A8127117504274047E60
:10A54F0000A807088005C333CE33CED8F9FF90FE9D
:10A55F00F3E0FDEF5D90FCE0600E127168126F4E3C
:10A56F00127073127951800C127168126F4E127043
:10A57F0073127AB81270FE700312710502A54702AA
:02A58F00B166B3
:10A4970090FE58EDF090FE55126FA1126F887D0760
:10A4A700128B2990FE55126F4E126FDB30E7149016
:10A4B700FE58E05403FFE52254036F6026E522545B
:10A4C700FC801290FE58E05401FFE52254016F60B2
:10A4D70012E52254FE4FF52212195F126F8C7D0789
:04A4E700128B292289
:10A8930090FE1EEBF090FE1CEFF0A3EDF0EF126FB5
:10A8A3008B128B2990FE1FE07002A3E0600D1271E2
:10A8B300998002C333D8FC4222800C127199800222
:10A8C300C333D8FCF4522290FE1CE0FFA3E0FD1238
:05A8D3006F8D028B29CE
:10A38A0090FE59EFF0ED1270F690FE59E0126FADA3
:10A39A0004F07D06FC1288C1EF7004E52260187F84
:10A3AA000112B5D990FE5CE004F0700690FE5BE005
:10A3BA0004F012717640D212717640107BFF7A3621
:10A3CA0079D290FE59E0126FC012A71E90FE59E092
:10A3DA00FF7B017AFE795A126FE804F07D06FC02CF
:02A3EA0088C128
:108B290090FD95EF126F9C1270EF90FD95E030E08B
:108B39002614FD7B017AFD7996127002128BE912D7
:108B49007087C00690FD95E0FD90FD97126F4E125B
:108B59007064E4A3F0802990FD95E0FD7B017AFD26
:108B69007996127002128BE9127087C00690FD95F2
:108B7900E0FD90FD97126F4E127064A37402F0E449
:108B8900FF1277A6D0E04F90FCDBF090FCDBE060B1
:108B99002390FCDFA3E0FF12B5CD12712894804029
:108BA90003127184127136700312713D12714450AF
:108BB90003028B3390FCDBE0FF601F7BFF7A367981
:108BC900FB126FC190FD9512701890FD96E0FF9011
:108BD900FBCEE4F0A3EFF012A71E90FCDBE0FF222E
:0A8BE90004F0A3F0E4FF1277A622C7
:1088C10090FD53EFF0A3EC126F9C1270EF90FD53EB
:1088D100E030E02614FD7B017AFD7954127002121A
:1088E1008986127087C00690FD53E0FD90FD5612F7
:1088F1006F4E127064E4A3F0802990FD53E0FD7B7C
:10890100017AFD7954127002128986127087C006AD
:1089110090FD53E0FD90FD56126F4E127064A374EA
:1089210002F0E4FF1277A6D0E04F90FCDBF090FC60
:10893100DBE0602390FCDFA3E0FF12B5CD127128CC
:1089410094804003127184127136700312713D12CA
:10895100714450030288CE90FCDBE0FF60217BFF75
:108961007A3679FB126FC190FD5312701890FD5445
:10897100E0FFA3E090FBCECFF0A3EFF012A71E9093
:10898100FCDBE0FF227402F0A314F0E4FF1277A6EF
:0189910022C3
:10A25F0090FEE2EEF0A3EFF0ED30E013786506E646
:10A26F001870010690FCDC126F4EF97864803A90FA
:10A27F00FEE2E07002A3E0703C786CA6B5ED540EE0
:10A28F007864760008F618E6FE08E67807C333CE42
:10A29F0033CED8F9FF786CE6FDEE7864F6EF4D0813
:10A2AF00F690FCDC126F4EF918E6FE08E612702BE2
:06A2BF00F5B475B20122A6
:04004E0078680622A6
:0C8E790041FC230041FC2A0F41FC2B00AF
:1071B50090FE0AE0FBA3E0FAA3E02404F9E43AFA1E
:1071C50012195F54FD1219C790FE0AE0FBA3E0FAFD
:1071D500A3E0F92290FC2FEFF090FC28E0FF7E0061
:1071E50078307CFC7D017B017AFF79821219399018
:1071F500FE0DE0FBA3E0FAA3E02403F9E43AFA026A
:10720500195F90FE04E0FBA3E0FAA3E022900015CD
:10721500121978FD2290FC27F0740FA3F0E490FC7E
:107225002FF090FC28E0FF7E0078307CFC7D017B10
:10723500017AFF79822290001C021E46740B90FD94
:107245003EF0E4A3F0A304F0A374FCF0A3742FF0C4
:1072550022900016021E46900009121E46EA494B6E
:1072650022EBF0A3EAF0A3E9F02290FC27F0A37447
:1072750002F090FC2AE090FC2FF090FF82E090FC59
:1072850030F02290001FE4F5F0021B9590FD2B7461
:1072950001F0A374FCF0A37431F022900009121ED2
:1072A5004602195FE490FC29F090FC2722121E4645
:1072B500900004021978900019021E4690001FE400
:1072C50075F001121AFCFEC3E5F02290FDE374018E
:1072D500F0A374FCF0A37424F02290FC27F0740151
:1072E500A3F090FC2AE090FC2F2290FD4E7401F053
:1072F500A374FFF0A37480F0221219D97B007A00E1
:10730500790022A37401F0A374FCF0A374402290C9
:10731500000102197890000202197890FF82E0FFBF
:1073250090FC30F07E0078317CFC7D017B017AFF9A
:10733500798322F0A37401F0E490FC2FF090FECA4B
:107345002290FC9DF090FC9A7401F0A374FAF0A3CE
:107355007496F090FC2C2290FC27E090FD3EF09076
:10736500FC28E090FD3FF0A3740122900003021970
:10737500781219C790FE042290FC27F07401A3F03F
:1073850090FF92E02254FD1219C790FECA22900088
:1073950001E40219D990001F121AC4C32212193927
:1073A50090FECA2290000502197890001FE475F03E
:1073B50064121B95740722121E46E9240122121E2F
:1073C50046E9240222900002E40219D9F090FF82D6
:1073D500E0240390FC28F0229000150219787B0127
:0573E5007AFA799622FE
:10AE150090FDF812726690FDF8E0F9A3E0FAA3E060
:10AE250090FC2CC912726790FDFBE0F9A3E0FAA330
:10AE3500E090FDBFC912726790FDF81271D0028AC9
:01AE45005FAD
:10837E0090FEC712726690FEC71271D0E41219C732
:10838E0090FEC71271D01273931273CA900003E459
:10839E001219D990000474401219D9900005E412F4
:1083AE0072FEC003C002C00190FEC71271D09000D1
:1083BE0006121E76127301C003C002C00190FEC7E2
:1083CE001271D0900009121E76127301C003C00202
:1083DE00C00190FEC71271D090000C121E7612735F
:1083EE0001C003C002C00190FEC71271D090000FF1
:1083FE00121E76127301C003C002C00190FEC71296
:10840E0071D0900012121E7690FEC71271D090009D
:10841E0015ED1272FEC003C002C00190FEC71271AC
:10842E00D0900016121E76127301C003C002C00156
:10843E0090FEC71271D0900019121E76127301C0F1
:10844E0003C002C00190FEC71271D090001C121E14
:10845E007690FEC71271D090001FE4F5F0021B95C6
:06B64B0090FC23EFF02249
:1087140090FCF312726690FCF91271D0C003C0028F
:10872400C00190FCF61271D0900009121E7690FCE4
:10873400FC1271D0C003C002C00190FCF61271D0CB
:1087440090000C121E7690FCF91271D0EA494B602D
:108754001690FCF61271D0C003C002C001A31271BE
:10876400D0900006121E7690FCFC1271D0EA494BA0
:10877400601890FCF61271D0C003C002C00190FCD6
:10878400FC1271D0900006121E7690FCF31271D088
:10879400C003C002C001A31271D0900019121E764A
:1087A40090FCF91271D0EA494B601890FCF31271F5
:1087B400D0C003C002C00190FCF91271D090001621
:1087C400121E7690FCFC1271D0EA494B601890FCA2
:1087D400F31271D0C003C002C00190FCFC1271D02E
:0787E400900016121E762220
:108F0F0090FCFF12726690FD051271D0C003C00273
:108F1F00C00190FD021271D090000F121E7690FDCD
:108F2F00081271D0C003C002C00190FD021271D0AF
:108F3F00900012121E7690FD051271D0EA494B6017
:108F4F001690FD021271D0C003C002C001A31271AE
:108F5F00D0900006121E7690FD081271D0EA494B90
:108F6F00601890FD021271D0C003C002C00190FDC5
:108F7F00081271D0900006121E7690FD051271D066
:108F8F00EA494B601890FCFF1271D0C003C002C0B9
:108F9F000190FD051271D0900016121E7690FD08FB
:108FAF001271D0EA494B601890FCFF1271D0C003C8
:108FBF00C002C00190FD081271D0900016121E76EB
:018FCF00227F
:10B50300C003C002C00190FE011271D090001C1252
:03B513001E76227F
:1037F10090FECA12726690FECA1271D012940850DD
:103801002590FC2C1271D0123D881271D01272BB1E
:10381100123D9E12720A240412720012738A1271EE
:10382100D074011219C790FECA1271D012731430EC
:10383100E61E1273937D40128CBC90FECA12720A6E
:10384100240412720012738A1271D074011219C702
:1038510090FECA1271D012195F14604D14607B146E
:10386100700302391224FE700302394824056003F3
:10387100023A0990FC2C1271D0123D881271D012BB
:1038810072BB123D9E1271D012723BE4FD12846E26
:1038910090FECA1271D012723B7D0112A44290FEB9
:1038A100CA1271D07401023A0690FECA1271D01286
:1038B1009CCC4003023A0990FECA1271D012728860
:1038C10012B4F090FECA1271D01272BB12AEA29065
:1038D100FECA1271D07402023A0690FECA1271D069
:1038E100129726502A90FECA1271D01272C19419F1
:1038F100EE94005003023A091272881272BB129EB2
:103901005812B52990FECA1271D07403023A06808A
:103911002A90FECA1271D01272BB12ADE3EF601B86
:1039210090FECA1271D01272C19432EE940050030B
:10393100023A091272887405023A0690FECA12719F
:10394100D0127288023A0990FECA1271D01272BB6B
:1039510012B5A7EF601490FECA1271D01272BB1299
:10396100B446EF90FECA6020801290FECA1271D058
:103971001272BB12B446EF90FECA600C12720A2496
:10398100041272004402800A12720A2404127200A4
:1039910054FD1219C790FECA1271D012739A942C59
:1039A100E5F09401500A90001FE475F001121B48E4
:1039B1001272BB12ADE3EF704F90FECA1271D012BA
:1039C100739A942CE5F09401402E1272B530E113F4
:1039D10012AE7690FECA12720A240412720054FDCD
:1039E1001219C790FECA1271D07D80128CBC90FE54
:1039F100CA1271D07402800D90FECA12720A240498
:103A010012720054FD1219C790FECA1271D01272BF
:103A11003B129C464003023C4E90FECA1271D012EA
:103A2100723B1272EFA3E4F0A37413F012A9E090B9
:103A3100FF80E0B410004003023C4E903A43F82866
:103A41002873023A73023A94023A9B023AA2023A6A
:103A5100AD023ABD023AD1023AF6023B0C023B21D9
:103A6100023B31023B46023B5F023B75023B850252
:103A71003BA41272A9041273D190FF92E0B40F0813
:103A810090FC2F740FF08005E490FC2FF01273204E
:103A9100023B011272A9741980171272A9741A805B
:103AA1001090FECA1271D07D04023C4B1272A974AF
:103AB1001C1273381271D07D40023C4B1272A974F2
:103AC10006F0E4A3F090FECA1271D07D40023C4B97
:103AD10078247CFC1272327E007F031273A2127171
:103AE100D012723B1272D012AD4690FECA1271D042
:103AF1007D10023C4B1272A97410F0A314127221B2
:103B01001273A21271D07D40023C4BE490FC29F06B
:103B1100741212721A1273A21271D07D40023C4BC0
:103B21001272A974131273381271D07D40023C4B8A
:103B3100E490FC29F0741D12721A1273A21271D052
:103B41007D40023C4B1272A9741EF0A37402F0E492
:103B510012727B90FECA1271D07D40023C4B1272F0
:103B6100A97415F074061272201273A21271D07D1D
:103B710040023C4B1272A974161273381271D07D37
:103B810040023C4B90FC297401F090FC27741FF01B
:103B9100A37402F0E412727B90FECA1271D07D40D0
:103BA100023C4B90FF8112727A90FC2FE064057009
:103BB10047A3E0702390FECA1271D012723B90FDB0
:103BC100E912729412A328EF6003023C4E90FECAE0
:103BD1001271D07D80023C4B90FECA1271D01272DC
:103BE1003B90FDE912729412A328EF606090FECA27
:103BF1001271D07D80023C4B90FC30E0702190FE30
:103C0100CA1271D012723B90FD3412729412730871
:103C1100123D92703890FECA1271D07D80802B9037
:103C2100FECA1271D012723B90FD3412729412735B
:103C310008123D92601790FC2FE0FF90FC2AE0B53E
:103C4100070B90FECA1271D07D80129BBE90FECAF6
:103C51001271D012731AFD600C129BBE90FECA1233
:103C610071D01273CA90FECA1271D012737030E310
:103C710028E91271FE54F712738C1271D012723B43
:103C8100C0037406127243D003E4FD12A12790FE13
:103C9100CA1271D07D08029BBE90FECA1271D01269
:103CA100737030E42EE91271FE54EF12738C1271AD
:103CB100D012723B1272D012AD4690FECA1271D070
:103CC10012723BC00390FD3E740CF0E4A3F0A30418
:103CD100023D7D90FECA1271D012737030E63CE94C
:103CE1001271FE54BF1219C790FC27E0B4071A9055
:103CF100FECA1271D012723B90FDF57401F0A374EB
:103D0100FCF0A37430F012AD7B90FECA1271D01298
:103D1100723B12735C12724C023D8290FECA1271A8
:103D2100D012737030E517E91271FE54DF12738CF3
:103D31001271D012723B90FC2AE0FD029F5590FE59
:103D4100CA1271D012737030E73CE91271FE547FD0
:103D51001219C71272A97418F0A37402F090FC2F03
:103D610014F0E4A3F090FECA1271D012723BC003AA
:103D710090FD3E7418F0A37402F0A31412724CD09B
:103D810003E4FD12A1272212B04F12B4F090FECA33
:103D910022F0128BF390FC2AEFF0640F2212AEA2F4
:043DA10090FECA22A4
:1057DB0090FE04127266900006121E4690FE07128F
:1057EB00726690FE041271D0129408400E90FE0463
:1057FB001271D012731470030258D790FE041271F9
:10580B00D0127256C003C002C00190FE041271D0B8
:10581B00127212D001D002D00312B30012720724FD
:10582B000412720054FD1273761271D0127256C0AC
:10583B0003C002C00190FE041271D0127212D0018B
:10584B00D002D00312B23B90FE041271D0127256EA
:10585B00C003C002C00190FE041271D0127212D0AC
:10586B0001D002D003125BD51271D01272BB12AEF3
:10587B00A290FE041271D012728812731430E70AD0
:10588B0090FE041271D07D80802190FE041271D0A5
:10589B0012731430E62290FE0712720A2401127260
:1058AB000044401273761271D07D40128CBC90FE76
:1058BB00041271D07402800890FE041271D074012E
:1058CB001219C790FE041271D012739390FE04123A
:1058DB0071D012195F147003025A90147003025A9C
:1058EB00A9147003025AC2147003025B35147003BF
:1058FB00025B3F24056003025B72127256C003C049
:10590B0002C00190FE041271D0127212D001D002AB
:10591B00D003125BD51271D01272BB12AEA290FEE5
:10592B00071271D012195F70411273A990FE0430E7
:10593B00E40C12720A24051272004410800A1272CF
:10594B000A240512720054EF1219C790FE07127148
:10595B00D01273A990FE0430E503025A3E12720A6C
:10596B00240512720054DF025A48127207240512E2
:10597B00720054EF1219C754DF1273761271D012E2
:10598B007256C003C002C00190FE041271D0127295
:10599B0012D001D002D00312B1F990FE041271D0D3
:1059AB001272BB129E5890FE041271D0127256C026
:1059BB0003C002C00190FE041271D0127212D0010A
:1059CB00D002D00312AA9BEF700D1272072405129E
:1059DB0072004410025A4890FE041271D012725693
:1059EB00C003C002C00190FE041271D0127212905B
:1059FB00FD7D1272F2D001D002D003129363EF70CF
:105A0B000C127207240512720044108030127207B8
:105A1B00240512720054EF1219C790FE041271D0B4
:105A2B001273DDFF7B017AFF7980129150EF7010BA
:105A3B0090FE0412720A240512720044200219C748
:105A4B00127207240512720054DF1219C790FE045C
:105A5B001271D0127256C003C002C00190FE041224
:105A6B0071D0127212D001D002D00312B2E090FEAC
:105A7B00041271D01272BB12AEA290FE041271D03E
:105A8B007401025B6D90FE041271D0129CCC40032A
:105A9B00025B7B90FE041271D07402025B6D90FE70
:105AAB00041271D01297264003025B7B90FE041206
:105ABB0071D07403025B6D90FE071271D012195FE7
:105ACB00D394035003025B7B90FE041271D01272CD
:105ADB00BB129E5890FE041271D0127256C003C0B6
:105AEB0002C00190FE041271D0127212D001D002CA
:105AFB00D00312B1F990FE041271D0127256C0038A
:105B0B00C002C00190FE041271D0127212D001D0EB
:105B1B0002D00312B27D12720724041272004401E8
:105B2B001273761271D07404803890FE041271D007
:105B3B007405802E90FE071271D01272B590FE0480
:105B4B0030E11512720A24041272004402127376A9
:105B5B001271D01273AF800A12720A2404127200EF
:105B6B0054FD1219C7800990FE041271D0124DD149
:105B7B0090FE041271D0129DD712720750092404A3
:105B8B0012720044108007240412720054EF121991
:105B9B00C790FE041271D012731AFD600C129BBEDB
:105BAB0090FE041271D01273CA90FE041271D012BF
:105BBB007370FF601490FE071271F74F1273761219
:105BCB0071D0900003E41219D92212B2E090FE04B6
:015BDB0022A7
:1023A10090FE0A127266900006121E4690FE0D12F1
:1023B10072661271CD12195FD39401500302248DFC
:1023C100127256C003C002C0011271CD127212D036
:1023D10001D002D00312A0BDEF60111271CD1272B3
:1023E100B520E508127314700302248D1271CD1209
:1023F1007256C003C002C0011271CD127212D00117
:10240100D002D00312B3001271B5127256C003C0CC
:1024110002C0011271CD127212D001D002D003128A
:10242100B23B1271CD127256C003C002C0011271CB
:10243100CD127212D001D002D00312B2E01271CDCE
:1024410012728812731430E72B1271CD127256C0BA
:1024510003C002C0011271CD127212D001D002D09C
:102461000312A0BDEF90FE0A60051271D0800E121A
:1024710071D0800D1271CD12731430E60474028094
:102481000274011219C71271CD1273931271CD1218
:10249100195FB4070040030229799024A2F8282883
:1024A100730224B70225EF02279F0227B7022829CA
:1024B10002283A022907127256C003C002C0011253
:1024C10071CD127212D001D002D00312B2E090FE8F
:1024D1000D1271D012195F704B1273A990FE0A3060
:1024E100E40C12720A24051272004410800A12725E
:1024F1000A240512720054EF1219C790FE0D1271D1
:10250100D01273A990FE0A30E50D12720A24051249
:10251100720044200225B012720A2405127200547E
:10252100DF0225B090FE0A12720A240512720054CD
:10253100EF1219C754DF1271CA127256C003C002DA
:10254100C0011271CD127212D001D002D00312B1AA
:10255100F91271CD127256C003C002C0011271CDC1
:10256100127212D001D002D00312AA9BEF700F9009
:10257100FE0A12720A24051272004410803112718F
:10258100CD127256C003C002C0011271CD12721277
:1025910090FD7D1272F2D001D002D003129363EF4D
:1025A100701090FE0A12720A240512720044100281
:1025B10019C790FE0A12720A240512720054EF1212
:1025C10019C71271CD127256C003C002C001127137
:1025D100CD127212D001D002D00312B2E01271CD2D
:1025E10012723B7D0412846E1271CD022A0E127199
:1025F100CD127256C003C002C0011271CD12721207
:10260100D001D002D00312A0BDEF7003022A1B1229
:1026110071CD1272B530E503022A1B90001FE475DB
:10262100F001121AFCFCC3E5F0940AEC940050038B
:10263100022A1BEFB4021D12739A9464E5F0940010
:102641005003022A1B90FE0D12720A24041272001A
:10265100547F800D90FE0D12720A24041272004400
:10266100801219C71271CD1273DDFF1273E3127359
:10267100EAEF601B1271CD12739A9419E5F0940080
:102681005003022A1BE924051272004440800D9078
:10269100FE0A12720A240512720054BF1219C712DF
:1026A10071CD1272881273E3129A18EF90FE0A60CC
:1026B1004B12720A240412720044011219C71273D8
:1026C100E312A191749A2FF974FA3EFA90FDDD7428
:1026D100011272671271CD12723B12AD111271CDDE
:1026E10012723B7D0212A4421271CD12723BC003E1
:1026F100127241D003E4FD12A127800D12720A2447
:102701000412720054FE1219C71271CD12723BE904
:102711004A4B60381271CD12723B12731430E02CA7
:102721001271CD12725612B5A7EF600D1271CD1252
:1027310072B530E6047F0180027F00EF440412731A
:10274100461271D0120280EF604F803D1271CD129E
:10275100725612B5A7EF600D1271CD1272B530E647
:10276100047F0180027F001271CD1273DDFE90FCA7
:1027710023E0B506047E0280027E00EE4F1273460E
:102781001271D0120280EF601090FE0D12720A24B5
:102791000112720044401219C71271CD80131271D7
:1027A100CD1272C1940AEE94005003022A1B1272D8
:1027B100887403022A1090FE0D1271D012195FD392
:1027C10094035003022A1B1271CD1272B530E01A24
:1027D100127256C003C002C0011271CD127212D022
:1027E10001D002D00312B27D801B1271CD1272563C
:1027F100C003C002C0011271CD127212D001D00209
:10280100D00312B3201271CD127256C003C002C0A0
:10281100011271CD127212D001D002D00312B1F99E
:102821001271CD7404022A101271CD12725612ABBC
:102831008D1271CD7405022A101271CD127256C01B
:1028410003C002C0011271CD127212D001D002D0A8
:1028510003120026EF70261271CD127256C003C00A
:1028610002C0011271CD127212D001D002D0031236
:10287100B2E01271CD1272887406022A101271CD63
:10288100127256C003C002C0011271CD127212D071
:1028910001D002D00312A0BDEF6401704190FE0D82
:1028A1001271D01272B520E7261271CD127256C084
:1028B10003C002C0011271CD127212D001D002D038
:1028C1000312B2E01271CD12728874011219C7900D
:1028D100FE0D12720A24041272004480800D90FED3
:1028E1000D12720A2404127200547F1219C790FE4D
:1028F1000D1271D01272B520E103022A1B1271CDA3
:102901001273AF022A101271CD1272C194FAEE94B1
:10291100005003022A1B127288127256C003C002B1
:10292100C0011271CD127212D001D002D00312B1C6
:10293100F912B1661271CD127256C003C002C00104
:102941001271CD127212D001D002D003120026EF03
:1029510060081271CD74031219C71271CD1272562B
:10296100C003C002C0011271CD127212D001D00297
:10297100D00312B2E0022A1B1271CD127256C003AB
:10298100C002C0011271CD127212D001D002D00367
:10299100120026EF60201271CD127256C003C002E0
:1029A100C0011271CD127212D001D002D00312A057
:1029B100BDEF6401605E1271CD127256C003C00298
:1029C100C0011271CD127212D001D002D00312B324
:1029D100001271B5127256C003C002C0011271CD4E
:1029E100127212D001D002D00312B23B1271CD1279
:1029F1007256C003C002C0011271CD127212D00111
:102A0100D002D00312B2E01271CD12728874011299
:102A110019C780061271CD124DD11271CD12195FF5
:102A2100FF640C6019EFD394024013EF6406600E4B
:102A310090FA90E020E70790FA8FE030E30AE9246A
:102A4100041272004410800D90FE0A12720A2404CE
:102A510012720054EF1219C71271CD12723B129CFF
:102A6100464003022CB21271CD12723B1272EFA3D7
:102A7100E4F0A37413F012A9E090FF80E0121ECFDE
:102A81002AC1002B01032B0C052B14062B36072B17
:102A91005E082B7D092B9B0C2BBD0D2BEC102BF411
:102AA100112C09122C17132C32142C17152C431628
:102AB1002C50172C5D182C70192C7F1A00002CB289
:102AC10090FF92E0FDB405047E0180027E0090FC3F
:102AD10029EEF090FC2774011273D1EDB405089032
:102AE100FC2F7405F0801390FF92E0B40F0890FC66
:102AF1002F740FF080041272E7F0127320022B562C
:102B010090FC27741BF0E4A3022B921271F4440889
:102B1100022CAF78247CFC1272327E007F031219E2
:102B2100391271CD12723B1272D012AD461271F48C
:102B31004410022CAF90FC277410F0A314F090FF06
:102B410092E0B405047F05800590FC2AE0FF90FC2B
:102B51002FEF1272261271F14440022CAF90FC2724
:102B61007412F0740F127383B405047F058005900D
:102B7100FC2AE0FF1271D94440022CAF7413127386
:102B81007DB405047F05800590FC2AE0FF90FC2FB1
:102B9100EFF01271F44440022CAF90FC277415F051
:102BA100A37406F090FF92E0B405047F05800590C0
:102BB100FC2AE0FF1271D94440022CAF7416127343
:102BC1007DFFB405047E05800590FC2AE0FE90FCA3
:102BD1002FEEF01271F444401219C7EF640560033F
:102BE100022CB21271F44480022CAF1271F4442011
:102BF100022CAF74071272DFF012722E7E007F0872
:102C01001271F14440022CAF74081272DFF012719C
:102C1100F44440022CAF90FC277409F07411127235
:102C2100E5F012722E7E007F101271F14440022CE9
:102C3100AF78407CFC1272327E007F0E121939028D
:102C41002CB2741412726F1271F44440022CAF74DE
:102C51000D12726F1271F44440022CAF90FC277474
:102C61000EF0A374091272E61271DD4440803F90A8
:102C7100FC27740F1272721271F44440803090FC80
:102C8100277417F0A37403F090FC2F740512727E61
:102C910090FF84E0600790FC2AE0FF80027F0090B3
:102CA100FC31EFF01271F444401219C7448012193B
:102CB100C71271CD12731A30E127E9240212720092
:102CC10054FD1219C7E490FC2FF01271CD12723B22
:102CD10090FD3E741AF0A37401F0A312724C022EFF
:102CE100161271CD12731A30E21DE924021272001C
:102CF10054FB1271CA12723BC00390FD3E741B1249
:102D01007246D003022E161271CD12731A30E31DD2
:102D1100E9240212720054F71271CA12723BC00305
:102D210090FD3E7406127246D003022E161271CD2A
:102D310012731A30E429E9240212720054EF12715D
:102D4100CA12723B1272D012AD461271CD12723B91
:102D5100C00390FD3E740C127246D003022E16126F
:102D610071CD12731A30E61CE9240212720054BFAD
:102D71001271CA12723B90FC29E0FD12735C12724F
:102D81004C022E491271CD12731A20E703022E5CF8
:102D9100E92402127200547F1219C790FC2FE064DB
:102DA100057042A3E0640470151271CD12723B12DA
:102DB1007291A3E4F0A3F0A3F0127EDD800A90FCEF
:102DC10030E0700FA374FFF01271CD12723B7D02DF
:102DD10002A4421271CD12723B127291A3E4F0A3CC
:102DE100F0A3022E5890FC30E06404702C1271CDD7
:102DF10012723B127291127308F0127EDD1271CDC4
:102E010012723B7D0212A4421271CD12723BC003B9
:102E1100127241D003E4FD802F90FC30E0702CA3AE
:102E21007404F01271CD12723B7D0412846E127122
:102E3100CD12723B7D0212A4421271CD12723BC0BF
:102E410003127241D003E4FD02A1271271CD127267
:0C2E51003B127291127308F0127EDD2219
:0BB5FD00E9240412720044200219C768
:0BB60800E9240412720054DF0219C78D
:1094080090FECD12726690FECD1271D012195FD304
:1094180094014003D38001C340012212725C60139F
:1094280090FECD1271D01272A0B40103D38001C393
:1094380040012290FECD1271D090000C12725F6034
:109448001690FECD1271D090000C1272A3B40103D5
:10945800D38001C340012290FECD1271D090000F3D
:1094680012725F601690FECD1271D090000F1272CA
:10947800A3B40103D38001C340012290FECD127131
:10948800D090001212725F601690FECD1271D090CB
:1094980000121272A3B40103D38001C3400122D386
:0194A80022A1
:109CCC0090FED012726690FED01271D012725C604F
:109CDC001090FED01271D01272A0D394014002D316
:109CEC002290FED01271D090000C12725F60139013
:109CFC00FED01271D090000C1272A3D394014002CA
:109D0C00D32290FED01271D090000F12725F6013AC
:109D1C0090FED01271D090000F1272A3D394014018
:109D2C0002D32290FED01271D090001212725F609A
:109D3C001390FED01271D09000121272A3D3940122
:069D4C004002D322C322F5
:1097260090FED312726690FED31271D012725C60F4
:109736001590FED31271D01272A0FF64036007EF7A
:10974600D3940140012290FED31271D090000C12E6
:10975600725F601890FED31271D090000C1272A343
:10976600FF64036007EFD3940140012290FED312F9
:1097760071D090000F12725F601890FED31271D0F4
:1097860090000F1272A3FF64036007EFD3940140A9
:10979600012290FED31271D090001212725F6018EF
:1097A60090FED31271D09000121272A3FF64036070
:0A97B60007EFD39401400122D322F3
:109DD70090FED612726690FED61271D012725C6037
:109DE7001190FED61271D09000091272B220E402CF
:109DF700C32290FED61271D090000C12725F6011D0
:109E070090FED61271D090000C1272B220E402C3F9
:109E17002290FED61271D090000F12725F601190DF
:109E2700FED61271D090000F1272B220E402C32244
:109E370090FED61271D090001212725F601190FEE0
:109E4700D61271D09000121272B220E402C322D34C
:019E570022E8
:108CBC0090FED912726690FED91271D012725C605D
:108CCC002190FED91271D01272A0D394034013904C
:108CDC00FED91271D09000091273BC1272004D12A1
:108CEC0019C790FED91271D090000C12725F6024DB
:108CFC0090FED91271D090000C1272A3D394034041
:108D0C001390FED91271D090000C1273BC12720029
:108D1C004D1219C790FED91271D090000F12725FCC
:108D2C00602490FED91271D090000F1272A3D394CC
:108D3C0003401390FED91271D090000F1273BC1225
:108D4C0072004D1219C790FED91271D090001212F8
:108D5C00725F602490FED91271D09000121272A32F
:108D6C00D39403401390FED91271D0900012127359
:098D7C00BC1272004D1219C7224D
:109BBE0090FEDC12726690FEDC1271D012725C6046
:109BCE001390FEDC1271D09000091273C312720052
:109BDE004D1219C790FEDC1271D090000C12725FFC
:109BEE00601390FEDC1271D090000C1273C31272CF
:109BFE00004D1219C790FEDC1271D090000F127238
:109C0E005F601390FEDC1271D090000F1273C312BE
:109C1E0072004D1219C790FEDC1271D09000121214
:109C2E00725F601390FEDC1271D09000121273C33B
:089C3E001272004D1219C72239
:108E8500182F000000000000000000000000000096
:0A8E950000000000000000000000D3
:10A5910085128385138222860308E6FA08E64A4B70
:10A5A1002208E6FA08E6F9021EF5A3E0FEA3E0FFA1
:10A5B1002290FFFF121EFBEFF0C2A922AA06AB07F1
:10A5C10090FEF4E025E0227C00121A0DEF22F8A69D
:10A5D1000308A60208A60122F8E6FE08E6FFE4FC4D
:02A5E100FD2259
:10006E0090FFFF121EFBEBF090FFFE121EFBECF05A
:10007E00A3EDF012A5B2E58954FCFE12A591E0FBAA
:10008E004EF589900003121F1FE044C0F58B90FEC1
:10009E00F8E014605A147003020145240260030252
:1000AE00019712A59112A5ABEE54FE7009758C1630
:1000BE00EEC313EF805F12A59112A5ABEE54FC7048
:1000CE0010758C2DEF7802CEC313CE13D8F9020122
:1000DE008612A59112A5ABD394EAEE9415500B752A
:1000EE008CFC7D1612A5C8020186AF030201901288
:1000FE00A591A3E0FEEE700C758C0E12A591A3A334
:10010E00E0020186EE54FE700F758C1D12A591A3B0
:10011E00E0C313A3E013806012A59112A5ABD39494
:10012E00EFEE9410500A758CFE7D1112A5C8804812
:10013E0012A591E0FF804B12A591A3E0FEEE700B8D
:10014E00758C1012A591A3A3E0802DEE54FE700FB6
:10015E00758C2112A591A3E0C313A3E0138019128D
:10016E00A59112A5ABD394EFEE94105010758CFEA2
:10017E007C007D0F121A0DEF14F58D800C12A591D7
:10018E00E0FF12B35F7F00803CAF8C12A591E0FDC3
:10019E0025E02427F8760008A607AF8DED25E0248C
:1001AE0047F8760008A6077401A805088002C33335
:1001BE00D8FCF5887410A805088002C333D8FC4219
:0B01CE0089D2A97F01900004021EFBF3
:10B35F0012A5B212A591E0FF7410A807088002C3CE
:0EB36F0033D8FCF45289D2A9900001021EFBD3
:0BB61300EF75F003A4242F12A5CF2236
:0BB61E00EF75F003A4243B12A5CF221F
:108D850090FEF4EFF0FBC2A9E58954FC4BF589AFE1
:108D95008C7862760008A607AF8DE4FCFDFE785E50
:108DA500121DFDEB25E0244712A5D9785E121DC0E2
:108DB500C3EF9BFFEE9AFEED99FDEC98FCC004A96C
:108DC5000512A5BD242712A5D9D000121BC2C004C7
:108DD500C00512A5BD2428F9C3E7786396FF19E7F6
:108DE5001896FEE4FCFDD001D000EB2FFFEA3EFE15
:108DF500ED39FDEC38FC785E121DFD90FEF8E014AF
:108E0500601C14602424027033E47F19FEFDFC7895
:108E15005E121DC0121BC2E47B207A018014785EAD
:108E2500121DB4E47B0FFA8009785E121DB4E47B51
:108E350011FAF9F8121C4D785E121DFDD2A9786061
:068E4500E6FE08E6FF2234
:03000B0002863B2F
:10863B00C0E0C0F0C083C082C0D075D000C000C005
:10864B0001C002C003C004C005C006C007308812B9
:10865B00782F12A5986005782F12A5A275880102B4
:10866B0086F9308912783212A5986005783212A5F6
:10867B00A27588020286F9308A12783512A59860A5
:10868B0005783512A5A27588040286F9308B11780E
:10869B003812A5986005783812A5A2758808804E07
:1086AB00308C11783B12A5986005783B12A5A2750A
:1086BB008810803A308D11783E12A5986005783E6F
:1086CB0012A5A27588208026308E11784112A598AC
:1086DB006005784112A5A27588408012308F0F7803
:1086EB004412A5986005784412A5A2758880D0071E
:1086FB00D006D005D004D003D002D001D000D0D00A
:09870B00D082D083D0F0D0E0321E
:08B63300E5FF54077869F622D7
:0500060012B6330022D8
:10B37D0012B633E6FF700476098008EFB4010C783D
:0CB38D006976027869E660031680F822F9
:10B1D60012B633E6FF7004760C800FEFB4010678E2
:10B1E6006976048005EFB40209227869E6600316E1
:03B1F60080F822BC
:10B1660012B633E6FF700476178012EFB401067844
:10B176006976098008EFB4020C786976027869E688
:06B1860060031680F822B0
:10A6D10090FEF8E014601314602624027036E5FF42
:10A6E100540770387869760D802AE5FF54071460A5
:10A6F1000904702878697615801A786976038014C0
:10A70100E5FF54071460090470127869761A800411
:0DA71100786976057869E660031680F82205
:109ED70090FEF8E014602714604424027067E5FFE1
:109EE700540714600D146010240270617869764578
:109EF70080537869761B804D786976058047E5FF42
:109F0700540714600D146010240270417869765F5D
:109F1700803378697628802D7869760C8027E5FF6D
:109F270054071460101460131460162403701E780D
:109F370069766D80107869762F800A7869760F8048
:0E9F470004E47869F67869E660031680F82273
:10985900303204D2AED2BE90FEF8E014603014600B
:109869005624027079E5FF5407146010146013142C
:109879006016240370707869767E8062786976371D
:10988900805C786976138056786976018050E5FFA7
:109899005407146010146013146016240370477879
:1098A9006976A980397869764C80337869761E8023
:1098B9002D786976078027E5FF5407146010146036
:1098C900131460162403701E786976C080107869B5
:1098D9007658800A7869762480047869760A7869E6
:0798E900E660031680F8227F
:107C1F00303204D2AED2BE90FEF8E0146078147009
:107C2F0003027D0F24026003027D6EE5FF5407B44B
:107C3F0007004003027D7E907C4DF8282873027C5C
:107C4F0062027C69027C73027C7D027C87027C91DC
:107C5F00027C9B786A7603027D01786A760108764A
:107C6F0084027D6E786A76000876BC027D6E786A33
:107C7F007600087658027D6E786A760008762602BE
:107C8F007D6E786A760008760D027D6E786A7600D2
:107C9F00087601027D6EE5FF5407B407004003022A
:107CAF007D7E907CB8F8282873027CCD027CD702A9
:107CBF007CE1027CEB027CF4027CFD027D06786A9B
:107CCF007604087607027D6E786A76010876FD02E3
:107CDF007D6E786A76000876F9027D6E786A760096
:107CEF00087676807A786A76000876358071786AB9
:107CFF0076000876158068786A7600087604805FCB
:107D0F00E5FF5407B407005066907D1FF8282873CD
:107D1F00027D34027D3D027D46027D4C027D55027F
:107D2F007D5E027D67786A76040876898031786A8D
:107D3F00760208763E8028786A76018016786A7611
:107D4F00000876878019786A760008763D8010786B
:107D5F006A76000876198007786A760008760678C2
:107D6F006BE61846600908E6161870F31680F022C5
:10B55D007869760A7869E6166005127C1F80F522F7
:10B56D00786976647869E6166005127C1F80F5228D
:0CB5C100AE071FEE600512985980F522BD
:0CB5CD00AE071FEE6005127C1F80F52207
:0CB5D900AE071FEE600512B55D80F52284
:0CB5E500AE071FEE600512B56D80F52268
:108E9F000F4F000000000000000000000000000065
:018EAF0000C2
:10AFFB0090FFFF121EFBEFF08512838513822286D2
:10B00B000308E6FA08E64A4B2208E6FA08E6F902D4
:0AB01B001EF5E0FF7401A8070822EB
:10AA1F0090FFFF121EFBEDF012AFFB12B01D800274
:10AA2F00C333D8FC12B003F0E0FF42F312B003A31C
:10AA3F00E06005EF42F4800712B003E0F452F41225
:0FAA4F00B003E0F5F6D2A842F5900002021EFB1C
:10B3B50012AFFB12B01D8002C333D8FC12B003F0EC
:0AB3C500E055F2FF900001021EFBAC
:10B48A0012AFFB12B01D8002C333D8FCF452F59000
:05B49A000001021EFB91
:10B53B00EF75F003A4244FF8A60308A60208A60192
:01B54B0022DD
:0300030002954A19
:10954A00C0E0C0F0C083C082C0D075D000C000C0E7
:10955A0001C002C003C004C005C006C007E5F55536
:10956A00F6F523301811784F12B00A6005784F12B9
:10957A00B01475F601804E301911785212B00A6093
:10958A0005785212B01475F602803A301A117855DD
:10959A0012B00A6005785512B01475F604802630A8
:1095AA001B11785812B00A6005785812B01475F673
:1095BA00088012301C0F785B12B00A6005785B12C3
:1095CA00B01475F610D007D006D005D004D003D059
:1095DA0002D001D000D0D0D082D083D0F0D0E032F7
:088EB0000614000000000000A0
:1099870075BC01C390FCF1E094A890FCF0E09461F1
:1099970022781408E6FA08E6F5828A83021EF97827
:1099A70014860308E6FA08E64A4B2290FCEBE0FE31
:1099B700A3E0FF90FCEEE0FCA3E0FDC39FEC9E223A
:1099C700F5B7E490FCF0F0A3F022E5BC540690FC58
:1099D700F2F022ED5401C4333354C022781C080638
:1099E700E61886062224E4F582E434FEF583229005
:1099F700FCF0E004F02290FCF27403F022E490FC07
:109A0700EEF0A3F02290FCE8E0FBA3E0FAA3E0F974
:019A1700222C
:10ACDB00EF6019D2BAED6006D2B6D2B78004D2B407
:10ACEB00D2B543BB04E490FEE5F08017D2B9ED601A
:10ACFB0006D2B2D2B38004D2B0D2B143BB02E4903D
:06AD0B00FEE4F002AF7C43
:10AF7C00EF600543BB01800353BBFEEDB4020CEB49
:10AF8C005403C454F0FF1299DA800C1299DA4480FD
:0BAF9C00FFEB5403C454F04FF5B72244
:10AB150090FE5FEBF0EF6014D2BAED6006D2B6D2CC
:10AB2500B78004D2B4D2B543BB048012D2B9ED606C
:10AB350006D2B2D2B38004D2B0D2B143BB0212B1B5
:0CAB4500B290FE5FE0F5B3A3E0F5B6228D
:10B1B200E5BB54FE4FF5BBEDB402081299DB442EF9
:10B1C200F5B1221299DA44AEF5B175B4FF75B21F2A
:04B1D20043B1012262
:10B54C00EF75F003A42414F8A60308A60208A601BC
:01B55C0022CC
:1077A60090FCE6EFF0A3EDF0A3EBF0A3EAF0A3E97B
:1077B600F0129A04A3F0A3F0A3F090FCE6E0FE1208
:1077C60099ECE060037F012274E42E1299EE7401B5
:1077D600F0E5BB54FE4EF5BB75BC0190FCEDE02018
:1077E600E12E90FCE7E0F5BDE5B754F144021299AD
:1077F600C7E5BC20E00D12793D70031299F6129987
:107806008A40EE12998750051299D180031299FD8C
:1078160090FCF2E0600302792E90FCE7E020E003A2
:107826000278AC129A041299B240030278FF90FCD7
:10783600F2E060030278FFEF24FFFFEE34FFFEED77
:10784600B50715ECB5061190FCEDE020E00AE5B7AA
:1078560054F1440AF5B78008E5B754F14406F5B784
:107866001299C9E5BC20E00D12793D70031299F614
:1078760012998A40EE129A0C90FCEEE0FEA3E0F517
:10788600828E83E5BF1219D912998750051299D1B4
:1078960080031299FD90FCEFE004F0700690FCEE78
:1078A600E004F002782C129A041299B2504B90FC24
:1078B600F2E07045129A0C8D828C83121978F5BE0F
:1078C600E5B754F144061299C7E5BC20E00D1279DC
:1078D6004770031299F612998A40EE12998750055D
:1078E6001299D180031299FD90FCEFE004F0700626
:1078F60090FCEEE004F00278AF90FCEDE020E0288A
:10790600E5B754F1440E1299C7E5BC20E00D127993
:107916004770031299F612998A40EE12998750051C
:107926001299D180031299FD90FCE6E01299ECE4DD
:10793600F090FCF2E0FF2212000690FCF1E004F069
:0B7946002212000690FCF1E004F02289
:03004B0002920D11
:10920D00C0E0C0F0C083C082C0D075D000C000C027
:10921D0001C002C003C004C005C006C00790FEF522
:10922D00E5BBF053BBFEE5B230E1191299A6600F14
:10923D001299E370010614FF781AE6FD12999875DC
:10924D00B202804AE5B230E211781AE620E0064417
:10925D0001F675B20175B2048034E5B230E31078D1
:10926D001C7600087600781AA6B575B208801FE541
:10927D00B230E01A781AE6FD30E0131299A6600BB1
:10928D001299E370010614FF12999875B20190FEC0
:10929D00F5E0F5BBD007D006D005D004D003D00241
:0F92AD00D001D000D0D0D082D083D0F0D0E0322A
:0300530002909088
:10909000C0E0C0F0C083C082C0D075D000C000C0A6
:1090A00001C002C003C004C005C006C00790FEF6A0
:1090B000E5BBF0E5BB54FE4401F5BBE5B230E11F72
:1090C00078171299A86013781E1299E5700106149A
:1090D000FF781BE6FD781712999A75B2028050E569
:1090E000B230E211781BE620E0064401F675B201C9
:1090F00075B204803AE5B230E310781E7600087647
:1091000000781BA6B575B2088025E5B230E020785E
:109110001BE6FD30E01978171299A8600F781E122F
:1091200099E570010614FF781712999A75B20190AB
:10913000FEF6E0F5BBD007D006D005D004D003D0B2
:1091400002D001D000D0D0D082D083D0F0D0E03295
:10B0A100EBF0A3EAF0A3E9F02290FE30E0FBA3E08D
:10B0B100FAA3E0F92275A102439A03439C03539B2F
:09B0C100FC227B017AFF79802258
:1094A90090FE21EEF0A3EFF0A3EDF090FEF8E014AA
:1094B900600F146014240270507F007ED07D0280FA
:1094C9000E7F807EA97D0380067FB07E1E7D047C91
:1094D90000E5FF5407F9F8121CFFE47B20FAF9F8BC
:1094E90012A8D8C006C00790FE21E0FEA3E0FBAA9F
:1094F90006E4F9F8D007D00612A8D8C3E49F90FE75
:1095090025F074049E90FE24F0438780759850904E
:10951900FE24E0F5BAA3E0F5AA75A101E5A1B4011D
:109529000512B0B680037595037E007F127D007B1E
:10953900017AFC79C712227B90FE23E06002D2AC4B
:0195490022FF
:10A5E30090FE2612B0A1A3ECF0A3EDF0E4FFFE75FC
:10A5F300A101E5A1B4010512B0B68003759503D39B
:10A6030090FE2AE09FEE6480F890FE29E064809833
:10A61300401E90FE2612B0AD8F828E83121978F5FC
:10A6230099E59830E1FB5398FD0FBF00010E80CFF1
:01A633002204
:10B3E70090FEF7EFF07B017AFE79F77D017C001282
:08B3F700A5E390FEF7E0FF2240
:10AB510090FE2B12B0A1E4A3F0A3F090FE2B12B053
:10AB6100ADA3E0FEA3E0F5828E83121978FF601396
:10AB710012B3E790FE2FE004F070E090FE2EE004A7
:0CAB8100F080D890FE2EE0FEA3E0FF2242
:10A71E0090FBC712B0A190FBF27401F0A374FBF092
:10A72E00A374CAF090FBC7E0F9A3E0FAA3E090FE91
:10A73E0016C912B0A290FBF2E0F9A3E0FAA3E090E2
:10A74E00FE19C912B0A212B0C312A80312B0C312DE
:0DA75E00B49FAC06AD0712B0C312A5E322F4
:0300230002A4EB49
:10A4EB00C0E0C083C082C0D075D000C004C005C01E
:10A4FB0007E59830E02F90FCD7E0FF2401FDE43313
:10A50B00FCA3E06D7001EC601974C72FF582E43485
:10A51B00FCF583E599F090FCD7E004F0E0B4100271
:10A52B00E4F05398FED007D005D004D0D0D082D021
:04A53B0083D0E032B7
:10B0F1007FFF90FCD8E0FE90FCD7E06E601874C72B
:10B101002EF582E434FCF583E0FF90FCD8E004F0F6
:07B11100E0B41002E4F0229B
:10A3EC0090FE3012B0A1A3ECF0A3EDF0E4FDFCD391
:10A3FC0090FE34E09DEC6480F890FE33E06480982D
:10A40C00402F12B0F1EFF460F912B0AA8D828C8358
:10A41C00EF1219D9EFB40A12ED1D70011C12B0AA7B
:10A42C008D828C83E41219D980070DBD00010C803C
:06A43C00BEAE04AF0522D4
:108EB8004DFCB8000000FF000000000000F0E000DA
:108EC80041FCB40041FCB50041FCC50041FCC600B2
:088ED80041FCB70041FCB300AE
:109D5200C454F0FEEF4EFFF090FEDFE024B8F5822F
:109D6200E434FCF58322E0FF90FEE0E022E0FE9086
:109D7200FEEBE022E090FEE7FEE033333354F822BC
:109D820075A101E5A1640122E090FEE0FEE0C45469
:109D9200F0FD22E0FD90FEEBE0FCED6C22E0FF2402
:109DA200FB24FB22C454F0FD90FCB3E05DFDEE22E7
:109DB20090FEEBE0FFEE6F2290FEE0E0540FF0A386
:109DC200E0FF22E0FEC454F05FFFEE4FF022F4FE0B
:059DD200EF5EF0EE223F
:1069A70090FEE0EDF0A3EBF090FEDFEFF01460490E
:1069B700146079147003026A59147003026A782408
:1069C700FA7003026AAB147003026AF2240B6003C5
:1069D700026B5990FEE1E0FF700790FEE0E042FC99
:1069E70022EF90FEE0B40205E042C88004E0F452D2
:1069F700C890FEE0E0F452FC2290FEE1E0FF700751
:106A070090FEE0E042FD22EF90FCB4B40212129D2A
:106A170068FEEF4EFF90FCB4129D59E05F42FD22E5
:106A2700129D6890FCB4129DD052FD2290FEE1E0C9
:106A3700FF700790FEE0E042FE22EF90FEE0B40216
:106A470005E042D88004E0F452D890FEE0E0F4522A
:106A5700FE2290FEE1E07012129D5AC083C082129E
:106A67009D68FEEF4ED082D083F0129D5AE0F5B0BC
:106A77002290FEE1E0FF700790FEE0E042F322EF94
:106A870090FCB5B40212129D68FEEF4EFF90FCB564
:106A9700129D59E05F42F322129D6890FCB5129D4A
:106AA700D052F322129DBA7013129D5AC083C0822E
:106AB700129D8AEE4DD082D083F08028EF90FCC5DE
:106AC700B4020E129D6890FCC5129D52129DC5809E
:106AD70013129D68C454F0F4FEEF5E90FCC5129D3E
:106AE70059E05EF0129D5AE0F58A2290FEE0E054EC
:106AF7001CF0A3E0FF7018129D5AC083C082E0907B
:106B0700FEE0129D7AFDEE4DD082D083F0803CEFFF
:106B170090FCC6B40220129D6833333354F8FEEF5D
:106B27004EFF90FCC6129D59E0FE33333354F85F95
:106B3700FFEE4FF08015129D6833333354F8F4FE9F
:106B4700EF5E90FCC6129D59E05EF0129D5AE0F58B
:106B5700C122129D82706E90FEDF129D9F50072406
:106B6700FE602C026C8212B18C90FEE1E0FF700790
:106B770090FEE0E0429B22EF90FEE0B40205E04287
:106B87009C8004E0F4529C90FEE0E0F4529B22903B
:106B9700FEE1E0FF700790FEE0E0429722EF90FCF5
:106BA700B7B40212129D68FEEF4EFF90FCB7129D1C
:106BB70059E05F429722129D68F4FEEF5E90FCB7A2
:106BC700F0EE52972290FEDFE0FF24FA6033146064
:106BD7004214606124036003026C8290FEE1E0FED0
:106BE700700790FEE0E0429B22EE90FEE0B40205C3
:106BF700E0429C8004E0F4529C90FEE0E0F4529B5B
:106C07002290FEE1E090FEE07004E0429422E0F47E
:106C170052942290FEE1E0701574B82F129D60C067
:106C270083C082129D68FEEF4ED082D083F0129D02
:106C37005AE0F59522129DBA7013129D5AC083C06F
:106C470082129D8AEE4DD082D083F08028EF90FC8F
:106C5700B3B4020E129D6890FCB3129D52129DC5EB
:106C67008013129D68C454F0F4FEEF5E90FCB312DB
:0C6C77009D59E05EF0129D5AE0F5AD2240
:10B18C00EF24FA6011146012146013146014240478
:10B19C007013E4F5A12275A1012275A1022275A1FB
:06B1AC00032275A104223C
:1097C000AB05AA07EA14601914601B14601D14602D
:1097D0001F24FA6020146022240B7023E5805BFFB5
:1097E00022E5905BFF22E5A05BFF22E5B05BFF2254
:1097F000E5F25BFF22E58A5BFF22E5C15BFF2212F7
:109800009D827032EA24FB24FB500624FE600C800B
:1098100047AF0212B18CE59A5BFF22E58F5470FAD4
:10982000758F7090FCB6E591F0E4F58FE04591F00E
:109830008A8FE05BFF22EA24FA600F146011146043
:109840001324037013E59A5BFF22E5935BFF22E587
:09985000955BFF22E5AD5BFF22F0
:1079510090FEE6EFF0A3EDF090FEE6E0FF129D5EF3
:10796100E04DF0EF14602114603414603B14604268
:1079710024FA605414607B240B6003027A1A90FE8F
:10798100E6129D5DE0F5802290FEE7E0FF90FCB4F9
:10799100E05F42FD90FEE6129D5DE0F5902290FED3
:1079A100E6129D5DE0F5A02290FEE6129D5DE0F5F8
:1079B100B02290FEE7E0FF90FCB5E05F42F390FE5D
:1079C100E6129D5DE0F5F22290FEE6E0FF129D5E7B
:1079D100C083C082E090FEE7129D8E90FCC5E05D01
:1079E100FDEE4DD082D083F074B82F129D60E0F58A
:1079F1008A2290FEE6E0FF129D5EC083C082129D46
:107A010076FD90FCC6E05DFDEE4DD082D083F07432
:107A1100B82F129D60E0F5C122129D82704390FE45
:107A2100E6129D9F500724FE6010027AB712B18CB6
:107A310090FEE6129D5DE0F59A2290FEE6E0FF12CF
:107A41009D5EC083C082129D76FD90FCB7E05DFD16
:107A5100EE4DD082D083F074B82F129D60E0F59185
:107A61002290FEE6E0FF24FA601414601B146022E9
:107A71002403704274B82F129D60E0F59A2290FEA3
:107A8100E6129D5DE0F5932290FEE6129D5DE0F524
:107A9100952290FEE6E0FF129D5EC083C082E0FE6B
:107AA10090FEE7E0129DA64DD082D083F074B82FEE
:077AB100129D60E0F5AD221B
:107AB80090FEE8EFF0A3EDF090FEE8E0FF129D5E87
:107AC800E0FEEDF4FDEE5DF0EF1460211460351476
:107AD800603C14604324FA6056146077240B6003FA
:107AE800027B7E90FEE8129D5DE0F5802290FEE824
:107AF800129D5DE0F59090FEE9E0FF90FCB4E05F38
:107B0800F452FD2290FEE8129D5DE0F5A02290FE61
:107B1800E8129D5DE0F5B02290FEE8129D5DE0F56B
:107B2800F290FEE9E0FF90FCB5E05FF452F322909A
:107B3800FEE8E0FF129D5EE0FEF58A74B82F129D04
:107B480060C083C08290FEE9E0C454F0FF90FCC599
:107B5800027C1390FEE8E0FF129D5EE0FEF5C17422
:107B6800B82F129D60C083C08290FEE9129D7BFFF2
:107B780090FCC6027C13129D82703E90FEE8129D16
:107B88009F500724FE6010027C1E12B18C90FEE804
:107B9800129D5DE0F59A2290FEE8E0FF129D5EE0FE
:107BA800FEF59174B82F129D60C083C08290FEE9E3
:107BB800129D7BFF90FCB7805290FEE8E0FF24FA0C
:107BC800601414601B1460222403704A74B82F12C6
:107BD8009D60E0F59A2290FEE8129D5DE0F5932203
:107BE80090FEE8129D5DE0F5952290FEE8E0FF1218
:107BF8009D5EE0FEF5AD74B82F129D60C083C08213
:107C080090FEE9E0C454F0FF90FCB3E05FF4FFEEAF
:077C18005FD082D083F0224F
:106C830090FEEBEDF090FEEAEFF0146044146076B2
:106C9300147003026D2A147003026D4B24FA7003FF
:106CA300026D80147003026DD3240B6003026E2502
:106CB30090FEEAE0FF129D5EC083C082129D6FFDCD
:106CC300EE6DD082D083F074B82F129D60E0F58012
:106CD3002290FEEAE0FF129D5E129D6FFDF4FCEE32
:106CE3005CF59090FCB4E05D62FD74B82F129D607A
:106CF300C083C082129DB2D082D083F090FEEA128C
:106D03009D5DE0F5902290FEEAE0FF129D5EC08358
:106D1300C082129D6FFDEE6DD082D083F074B82FC8
:106D2300129D60E0F5A02290FEEAE0FF129D5EC096
:106D330083C082129D6FFDEE6DD082D083F074B854
:106D43002F129D60E0F5B02290FEEAE0FF129D5EF7
:106D5300129D6FFDF4FCEE5CF5F290FCB5E05D6214
:106D6300F374B82F129D60C083C082129DB2D0828B
:106D7300D083F090FEEA129D5DE0F5F22290FEEAE8
:106D8300E0FF129D5E129D6FF4FDEE5DF58A74B80F
:106D93002F129D60C083C08290FEEBE0C454F0FFCD
:106DA30090FCC5E05FFFEE6FD082D083F090FEEAE7
:106DB300E0FF129D5EC083C082129D6F540FFDEEF3
:106DC3006DD082D083F074B82F129D60E0F58A22D3
:106DD30090FEEAE0FF129D5E129D6FF4FDEE5DF5FD
:106DE300C174B82F129D60C083C08290FEEB129DC8
:106DF3007BFF90FCC6E05FFFEE6FD082D083F09004
:106E0300FEEAE0FF129D5EC083C082129D6F541C98
:106E1300FDEE6DD082D083F074B82F129D60E0F543
:106E2300C122129D82706890FEEA129D9F50072432
:106E3300FE6027026F3B12B18C90FEEAE0FF129DC9
:106E43005EC083C082129D6FFDEE6DD082D083F051
:106E530074B82F129D60E0F59A2290FEEAE0FF12CB
:106E63009D5E129D6FFDF4FCEE5CF59190FCB7E026
:106E73005D629774B82F129D60C083C082129DB269
:106E8300D082D083F090FEEA129D5DE0F5912290CE
:106E9300FEEAE0FF24FA602B1460461460612403C9
:106EA3006003026F3B90FEEAE0FE129D5EC083C06A
:106EB30082129D95D082D083F074B82E129D60E02B
:106EC300F59A2290FEEAE0FE129D5EC083C0821214
:106ED3009D95D082D083F074B82E129D60E0F59317
:106EE3002290FEEAE0FE129D5EC083C082129D9551
:106EF300D082D083F074B82E129D60E0F595227491
:106F0300B82F129D60C083C082129D6F129DA66D23
:106F1300D082D083F074B82F129D60C083C082E00A
:106F2300FF90FEEBE0540FFEEF6ED082D083F09023
:096F3300FEEA129D5DE0F5AD22BD
:10B3FF00786DE6FF90FF8093FE74802FF582E43422
:08B40F00FFF583EEF006E622D2
:10B45D00C3EE940240037FFF2274002FF58274EE39
:07B46D003EF583E493FF228A
:10A6340090FEECEEF0A3EFF0C3EE94025040748071
:10A644006480700374FFF4703530AF02D230C2AF4F
:10A6540090FEEDE0240090FEECE034EEF5F9A3E08A
:10A66400F5FA786D764012B3FFB480FAAF05786DD1
:0FA67400A6077B01796D12FFC0303002D2AF22F2
:10B0250074806480700374FFF4701E30AF02D230F8
:10B03500C2AF75F9EEE4F5FA786DF612B3FFB440D8
:0AB04500FA12FF80303002D2AF2271
:0C8EE000C13141FE610043FE6200000051
:10B3990090FE62E0FBA3E0FAA3E0F9EA494B2290B0
:0CB3A900FE62A3E0FAA3E0F5828A832292
:10ABC70075A101E5A1B4011BEF24FE600C14600E12
:10ABD7002403702375A49C801E75A4DC801975A4BA
:10ABE700FC801443F580EF24FE6009240270087589
:0AABF700A4B8800375A4F8D2BD22B3
:0CB5F10090FE62EBF0A3EAF0A3E9F02268
:10B1180030310CEF70037F862290FE61E0FF2275CC
:10B12800A101E5A1B40107EF04F5A6AFA722EF70CE
:07B1380003AFA622AFA7221E
:03006B0002A046AA
:10A04600C0E0C0F0C083C082C0D075D000C000C0E0
:10A0560001C002C003C004C005C006C007C23175F6
:10A06600A101E5A164017019F5A612B399602AE56C
:10A07600A530E6047F0180027F0012B3A8ADA78059
:10A086001512B3996013E5A530E6047F0180027FBF
:10A096000012B3A87D10121EF943A580D007D00682
:10A0A600D005D004D003D002D001D000D0D0D082C9
:07A0B600D083D0F0D0E032AE
:068EEC0041FEF801C13255
:06B6510090FEF8EFF0226C
:10B41700EF6005D232758680E5FFB430037F0122E5
:08B4270075FF30D2AF7F002257
:08B63B00303204D2AED2BE226F
:105BDC00444247434D4420537472696E67204275AA
:105BEC00666665722046756C6C0D0A00257320255F
:105BFC0058202558202558202558006275730044DC
:105C0C004247434D44206275733A204275733D30D0
:105C1C007825302E32582C20506F72743D307825F8
:105C2C00302E32582C2053706565643D3078253009
:105C3C002E32580D0A0063697200444247434D44AA
:105C4C00206369723A20436F64653D307825302EAD
:105C5C0032580D0A0077723000444247434D4420BD
:105C6C007772303A2049443D307825302E32582C0A
:105C7C00205265673D307825302E32582C204461F7
:105C8C0074613D307825302E32580D0A0072643024
:105C9C0000444247434D44207264303A2049443D0D
:105CAC00307825302E32582C205265673D307825BF
:105CBC00302E32582C20446174613D0030782530F0
:105CCC002E32580D0A0074623000444247434D4452
:105CDC00207462303A2049443D307825302E3258B9
:105CEC002C205265673D307825302E32582C204DB3
:105CFC0061736B3D307825302E32582C2044617402
:105D0C00613D0063623000444247434D442063626E
:105D1C00303A2049443D307825302E32582C2052D0
:105D2C0065673D307825302E32582C204D61736BD1
:105D3C003D307825302E32582C20446174613D0062
:105D4C0077723100444247434D44207772313A20F8
:105D5C0049443D307825302E32582C205265673D11
:105D6C00307825302E32582C20446174613D3078C7
:105D7C0025302E32580D0A007264310044424743DC
:105D8C004D44207264313A2049443D307825302E00
:105D9C0032582C205265673D307825302E32582CE5
:105DAC002053697A653D307825302E32582C2044AA
:105DBC006174613D002852656164206E756D626589
:105DCC0072206578636565642061206D6178206F51
:105DDC006620256420627974657329000D0A002001
:105DEC0000307825302E32582C200074623100445B
:105DFC004247434D44207462313A2049443D307847
:105E0C0025302E32582C205265673D307825302EA7
:105E1C0032582C204D61736B3D307825302E325822
:105E2C002C20446174613D0063623100444247435D
:105E3C004D44206362313A2049443D307825302E60
:105E4C0032582C205265673D307825302E32582C34
:105E5C00204D61736B3D307825302E32582C204408
:105E6C006174613D0077723200444247434D4420D7
:105E7C007772323A2049443D307825302E32582CF6
:105E8C00205265673D307825302E34582C204461E3
:105E9C0074613D307825302E32580D0A0072643210
:105EAC0000444247434D44207264323A2049443DF9
:105EBC00307825302E32582C205265673D307825AD
:105ECC00302E34582C2053697A653D307825302E8D
:105EDC0032582C20446174613D007462320044429B
:105EEC0047434D44207462323A2049443D30782572
:105EFC00302E32582C205265673D307825302E34A8
:105F0C00582C204D61736B3D307825302E32582C37
:105F1C0020446174613D0063623200444247434D4A
:105F2C0044206362323A2049443D307825302E3289
:105F3C00582C205265673D307825302E34582C2053
:105F4C004D61736B3D307825302E32582C204461D6
:105F5C0074613D004552524F523A204949432066E4
:105F6C0061696C65642025642C2049494341646453
:105F7C00723D307825302E32582C205265674164A2
:0D5F8C0064723D307825302E32580D0A0029
:088EF20041FC920041FC9000DC
:1075E900787E7CFC7D017BFF1220B4EF22787E7CC3
:1075F900FC7D017BFF1220B4EF22A3F090FC77E021
:10760900FF90FC7AE0FCA3E090FD61FD7B017AFC30
:10761900797EE4F0A304F022787E7CFC7D017BFF77
:107629001220B4EF22787E7CFC7D017BFF1220B40E
:10763900EF227BFF7A5D79ED90FC94E0247EF58260
:10764900E434FCF583E0FFE490FBCAF0A3EFF022F9
:10765900787E7CFC7D017BFF1220B4EF2290FC7EBA
:10766900F090FC77E0FF90FC79E0FD7B017AFC79F2
:107679007E22787E7CFC7D017BFF1220B4EF229074
:10768900FC79E0FEA3E04EF0A3E0F022E4F0A3745D
:1076990012F07BFF7A5D79C190FBCAE4F0A3741202
:1076A900F0227BFF7A5C79C890FC7EE0FF90FBCAF0
:1076B900E422F0A3EDF0A3EBF0A3EAF0A3E9F09044
:1076C900FC93E4F0A3740AF0E4A3F0A3F02290FC85
:1076D90079E0FD90FC7BE0FB22FDE0FBA3E0FAA34F
:1076E900E0F9A3E0FFA3E090FCEBCFF0A3EFF0ED0E
:1076F90022A3F0A37401F0A322A3F0A37422F04300
:10770900FF407AFF7980121EF553FFBF22E0FEA3E6
:10771900E0FF90FC93E0FCA3E0FDC39FEC9E22E018
:10772900FFE490FBCCF0A3EFF022D390FC94E0941B
:107739000090FC93E0940022C390FC96E09403909F
:10774900FC95E09400227BFF90FC76E0FFA3E02209
:10775900787E7CFC7D017BFF1220B4EF22E054FE91
:10776900FD7B0190FCEBE4F0A322A3E024FDF09063
:10777900FC93E034FFF02290FCEDEFF090FC90E0F8
:10778900FF227BFF7A5D79E82290FC7EE0FF90FC86
:0D7799007BE02290FC7EE0FF90FC7DE02272
:10432E0012B0F190FEF9EFF0F470030246F1E0FFE7
:10433E0090FC92E0FE04F0747E2EF582E434FCF5DF
:10434E0083EFF090FC92E0D39412400E7BFF7A5BE9
:10435E0079DC12A71EE490FC92F090FEF9E0FF6467
:10436E000A6008EF640D60030246F1E490FC92F0DF
:10437E0090FBF874FFF0A3745BF074F81276FA7485
:10438E00FFF074801276FA74FCF0A374761276FB4A
:10439E0074FCF0A374781276FB74FCF0A3747A129A
:1043AE0076FB74FCF0A3747CF012767412670EE444
:1043BE0090FC81F07A5C79071275E9701D7A5C7950
:1043CE000B1246F790FC77E0FF1276D712ACDB901B
:1043DE00FC77E090FC90F00246F17A5C794212751F
:1043EE00E9703F7A5C794612774FCF12765112A759
:1043FE001ED23190FC77E090FE61F090FE62E0FB01
:10440E00A3E0FAA3E0F9EA494B70030246F190FEED
:10441E0062A3A3E0F5828A837D10E4FF121EF902E7
:10442E0046F17A5C79611275F670127A5C796512D2
:10443E0046F71276D77F7512B5B40246F17A5C79DB
:10444E00991275F670207A5C799D12774F90FBCA9F
:10445E00CFF0A3EFF090FC78E0FFA3E0CF12772B24
:10446E0012A71E0244A67A5C79D212762170117AB6
:10447E005C79D612472A1276D77F6312B5B48018AC
:10448E007A5D790F12762170337A5D791312472A8D
:10449E001276D77F5312B5B490FC79E0FF12B516A1
:1044AE0090FC7CE4F0A3EFF07BFF7A5C79C890FC83
:1044BE007CE0FFA3E090FBCACF0246B27A5D794C56
:1044CE0012762E70247A5D795012475D90FC7BE057
:1044DE0090FC7EF090FC77E0FF90FC79E090FDA1DF
:1044EE001276141298F00246F17A5D798412762EC5
:1044FE0070777A5D798812475DD390FC7BE09412D9
:10450E0090FC7AE09400400612769512A71E90FC5D
:10451E0077E04401FFC00712766FA3E0FFA3E0909F
:10452E00FDA1CFF0A3EFF0D0071298F0EF600302D9
:10453E0046F190FC93F0A3F090FC7A127716502679
:10454E00ED540F700612778B12A71E90FC94E05458
:10455E0007700312486D12763B12487770DA90FCA2
:10456E0093E004F080D20246817A5D79F712765993
:10457E0070277A5D79FB1248131298F0EF600302F0
:10458E0046F1127792FEEF6E127666124860600365
:10459E000246F11276AB0246B27A5E793412765941
:1045AE0070287A5E79381248131298F0EF60030281
:1045BE0046F1127792F4FEEF5E1276661248606054
:1045CE00030246F11276AB0246B27A5E797112762A
:1045DE007B70171276887A5E797512479090FC7D03
:1045EE00E01276031296880246F17A5E79A9127667
:1045FE007B60030246871276887A5E79AD12479009
:10460E00D390FC7DE0941290FC7CE0940040061266
:10461E00769512A71E90FC77E04401FFC00790FC30
:10462E007AE0FCA3127672A3E0FFA3E090FD61CFC7
:10463E00F0A3EFF0D007129688EF60030246F190D8
:10464E00FC93F0A3F090FC7C1277165026ED540FDD
:10465E00700612778B12A71E90FC94E0540770031D
:10466E0012486D12763B12487770DA90FC93E00494
:10467E00F080D212778B0246EE7A5E79E612775987
:10468E0070291276887A5E79EA1247C3129688EFFD
:10469E00705112779CFEEF6E127603129688EF70B1
:1046AE00421276ABF0A3EFF00246EE7A5F79231258
:1046BE007759702F1276887A5F79271247C3129630
:1046CE0088EF701F12779CF4FEEF5E12760312963F
:1046DE0088EF700F7BFF7A5C79C890FC7E12764E65
:1046EE0012A71E90FEF9E0FF227BFF90FC76E0FF02
:1046FE00A3E090FBCACFF0A3EFF090FC78E0FFA30D
:10470E00E090FBCCCFF0A3EFF090FC7AE0FFA3E0BB
:10471E0090FBCECFF0A3EFF012A71E227BFF90FCF2
:10472E0076E0FFA3E090FBCACFF0A3EFF090FC7809
:10473E00E0FFA3E090FBCCCFF0A3EFF090FC7AE08B
:10474E00FFA3E090FBCECFF0A3EFF012A71E227BCB
:10475E00FF90FC76E0FFA3E090FBCACFF0A3EFF052
:10476E0090FC78E0FFA3E090FBCCCFF0A3EFF090AD
:10477E00FC7AE0FFA3E090FBCECFF0A3EFF012A700
:10478E001E227BFF90FC76E0FFA3E090FBCACFF0E9
:10479E00A3EFF090FC7AE0FFA3E090FBCCCFF0A368
:1047AE00EFF090FC7CE0FFA3E090FBCECFF0A3EF08
:1047BE00F012A71E227BFF90FC76E0FFA3E090FB99
:1047CE00CACFF0A3EFF090FC7AE0FFA3E090FBCC11
:1047DE00CFF0A3EFF090FC7CE0FFA3E090FBCECFF8
:1047EE00F0A3EFF012A71E90FC77E04401FF90FCBF
:1047FE007AE0FCA3E0FD7B017AFC797E90FD61E41A
:10480E00F0A304F0227BFF90FC76E0FFA3E090FB88
:10481E00CACFF0A3EFF090FC78E0FFA3E090FBCCC2
:10482E00CFF0A3EFF090FC7AE0FFA3E090FBCECFA9
:10483E00F0A3EFF012A71E90FC77E04401FF90FC6E
:10484E0079E0FD7B017AFC797E90FDA1E4F0A30472
:10485E00F02290FDA1E4F0A304F01298F0EF227B79
:10486E00FF7A5D79EB12A71E2212A71E90FC94E030
:03487E0004F02221
:1098F00090FD9CEF1276BB90FC90E0FF90FD9C7A6F
:10990000FD799D12776604F0A3F01277A690FC9182
:10991000EFF0E0FEC00690FD9CE090FD9E1276E226
:1099200030E0047F0080027F021277801277A6D099
:10993000E04F90FC91F0602390FC94E0FF12B5CDD5
:10994000127733400312777390FC96E004F07006B0
:1099500090FC95E004F0127741409C90FC91E0FF70
:10996000601F7BFF7A5F796012765090FD9C1277C2
:109970002890FD9DE0FF90FBCEE4F0A3EFF012A74E
:079980001E90FC91E0FF22A4
:1096880090FD5BEFF0A3EC1276BB90FC90E0FF90AE
:10969800FD5B7AFD795C1277667402F0A314F01210
:1096A80077A690FC91EFF0E0FEC00690FD5BE0909D
:1096B800FD5E1276E230E0047F0080027F021277BE
:1096C800801277A6D0E04F90FC91F0602390FC9434
:1096D800E0FF12B5CD127733400312777390FC96F2
:1096E800E004F0700690FC95E004F0127741409A8F
:1096F80090FC91E0FF60217BFF7A5F7960127650E1
:1097080090FD5B12772890FD5CE0FFA3E090FBCE14
:0E971800CFF0A3EFF012A71E90FC91E0FF220D
:10B5160090FF807485F0A3EFF0746E127702786E58
:03B52600E6FF221B
:0DB5B40090FF80EFF0A3EDF0EB1277022284
:0E8EFA0043FA8C01FA9641FA900041FA8F007B
:1087EB0090FE10E0FBA3E0FAA3E0F92290001FE457
:1087FB00F5F0121B95900015021978E0FEA3E0FF2F
:10880B007C007D051219FB90FA8CE0FBA3E0FAA328
:10881B00E02FF9EA3EA801FCAD037B017AFF7980DA
:10882B002290001FE4F5F0121B95900016021E46D5
:10883B0090FA90E0FFC390FA95E09F7480F890FA5D
:10884B0094E06480982290001FE475F001121AFCEA
:10885B00FEC3E5F02290FA90E075F005A4FF90FAC4
:10886B008CE0FBA3E0FAA3E022EBF0A3EAF0A3E990
:10887B00F022FD7401F0A374FFF0A37480F022903A
:10888B0000040219787E007F0512193990FA90E0E6
:10889B0004F0227F057E00122257EF2290FA90E01F
:1088AB004480F02290001FE4F5F0021B952404F99C
:0688BB00E43AFA02195F25
:104DD10090FE10128874900006121E4690FE131267
:104DE10088741287EB12195F24F9B407004003029B
:104DF1005301904E0175F003A4C58325F0C583735B
:104E0100024E16024EDD0250900250E602513F0260
:104E110051B902525590FE131287EE12888A30E181
:104E2100751287EB128835C003C002C0011287EBEF
:104E3100128800FDD001D002D00312B21A1287EB02
:104E41001288519464EE940050030253011287F7C3
:104E5100FF128825129150EF602A1287EB12888A7F
:104E610030E019128835C003C002C0011287EB126D
:104E71008800FDD001D002D00312B27D1287EB74FD
:104E8100080252FE1287EB128800FFE4FD12B0788F
:104E910090FE100250CA1287EB12888A30E0191274
:104EA1008835C003C002C0011287EB128800FDD013
:104EB10001D002D00312B27D1287EB128835C003F4
:104EC100C002C0011287EB128800FDD001D002D0D0
:104ED1000312B23B1287EB74050252FE1287EB12EA
:104EE1008800FFE4FD12B0781287EB12880012539C
:104EF1000290FE1030E61E1287EE128835C003C004
:104F010002C0011287EB128800FDD001D002D0034C
:104F110012B29E801C1287EE128835C003C002C0F7
:104F2100011287EB128800FDD001D002D00312B22A
:104F3100BFE490FF88F012A76B7C017D00121A621A
:104F410090FF88E02480F582E434FFF583EDF09052
:104F5100FF88E004F0E0C3940840DB1287EB12887D
:104F610035C003C002C0011287EB12880090FD76A4
:104F710012887DD001D002D00312AECE1287EB127F
:104F81008800FF1288251201D91287EB128835C0DB
:104F910003C002C0011287EB12880090FD7D1288C8
:104FA1007DD001D002D003129363EF70241287EBFE
:104FB100128835C003C002C0011287EB128800FDC0
:104FC100D001D002D00312B3201287EB7407025232
:104FD100FE1287EB128800FF12882512B0CA1287D1
:104FE100EB128800FF128825129150EF702412876E
:104FF100EB128835C003C002C0011287EB12880092
:10500100FDD001D002D00312B3201287EB74070246
:1050110052FE1287EB128835C003C002C00112870D
:10502100EB128800FD90FD8412887ED001D002D061
:105031000312AEFA1287EB900019121E46E94A4B91
:10504100704590FA90E0C394085039E490FA94F0D6
:10505100A3F012883B501812880612889E601090A7
:10506100FA95E004F070EB90FA94E004F080E3121A
:10507100883B40131288602FF9EA35F0128820121C
:10508100889080031288A71287EB74090252FE12DE
:1050910087EB1288519407EE9400500302530112DA
:1050A1008835C003C002C0011287EB128800FDD011
:1050B10001D002D00312AFA7EF90FE10600B128750
:1050C100EE1288AF740A0252FE1287EE128835C0C2
:1050D10003C002C0011287EB128800FDD001D0028B
:1050E100D00302B3201287EB12A1F8EF70311287BF
:1050F100EB128851940AEE94005003025301128876
:105101002CC003C002C0011287EB128800FDD00140
:10511100D002D00312B3201287EB74070252FE12A1
:1051210087EB1287F712530290FE1030E6081287C0
:10513100EE740D0252FE1287EE740B0252FEE490E1
:10514100FF80F01287EB12883512B58BEF700C904F
:10515100FF80E004F0E0C394FA40E8E490FF81F0BE
:105161001287EB12883512B58BBF010C90FF81E0DD
:1051710004F0E0C394FA40E81287EB128835C003CB
:10518100C002C0011287EB128800FDD001D002D00D
:105191000312B25C1287EB128835C003C002C00152
:1051A1001287EB128800FDD001D002D00312B23B6E
:1051B1001287EB740C0252FE90FE131287EE1288D6
:1051C1008A30E16C1287EB128851944BEE940050B7
:1051D100030253011288AF12A1F8EF70451287EB59
:1051E10012888A30E221128835C003C002C0011240
:1051F10087EB128800FDD001D002D00312B3001258
:1052010087EB74070252FE90FE1012886C1288B868
:1052110044041219C71287EB90001FE475F03202A3
:105221001B9590FE1012886C1288B854FB0252FE36
:105231001287EB128835C003C002C0011287EB123E
:105241008800FDD001D002D00312B3001287EB74A5
:10525100070252FE1287EB128800FF12B34090FA48
:1052610091EFF030E56C1287EB1287F7FF1288257A
:1052710012AC0190FF80E0FD20E71CA3E0FF20E3DA
:10528100161287EB90FD67EFF0127D7FEF60201221
:1052910087EB740B0252FE90FF80E030E703128827
:1052A100A790FF81E030E30790FA8FE04408F01205
:1052B10087EB128835C003C002C0011287EB128848
:1052C10000FDD001D002D00312B3201287EB740786
:1052D100802B1287EB12885194FAEE940040211230
:1052E100882CC003C002C0011287EB128800FDD0D8
:1052F10001D002D00312B3201287EB74071219C731
:0B53010022FF12B34090FA91EFF0225F
:10A1F80090FDA3128874128835C003C002C0019074
:10A20800FDA31287EE128800FD90FD8B7401F0A368
:10A2180074FDF0A374A6F0D001D002D00312A84DAB
:10A22800EF7002FF2290FDA31287EE128800FF7BD9
:10A23800017AFD79A812A2C5EF7002FF2290FDA84D
:10A24800E0FEA3E0FF90FDA6E0B50608A3E0B50791
:07A25800037F01227F0022B9
:107D7F0090FD63128874A3EDF0A3E0540FFF90FA07
:107D8F008FE0FEEFD39E40028002AF0690FA8FEF96
:107D9F00F012AAD8E490FA92F0A3F090FD66E0FFFB
:107DAF0090FA92E0FCA3E0FDC39F7480F8EC64802E
:107DBF00984003027E4590FD631287EE128800FF04
:107DCF0012882590FDD8EDF090FD66E090FDD9F07A
:107DDF00128262EF7002FF2290FA90E0C394085073
:107DEF0039E490FA94F0A3F012883B5018128806E9
:107DFF0012889E601090FA95E004F070EB90FA9460
:107E0F00E004F080E312883B40131288602FF9EAF8
:107E1F0035F012882012889080031288A7128825C7
:107E2F007D051292BC90FA93E004F0700690FA92DE
:107E3F00E004F0027DAA90FD66E0701890FD6312D9
:107E4F0087EE128800FF128825E490FDD8F0A30476
:107E5F00F012826290FD66E090FF80F090FD67E087
:107E6F0090FF81F090FD631287EE128835C003C03A
:107E7F0002C00190FD631287EE128800FD90FD9203
:107E8F007401F0A374FFF0A37482F0D001D002D07C
:107E9F000312AFD11288257D0A1292BC128556901B
:107EAF00FD6812887490FD631287EE128800FF122E
:107EBF00882512AC3890FD6812886CF8AC021288D5
:0E7ECF00237F141288A060037F00227F01220F
:068F080043FBAD01FFC0B8
:1089920090FBBBE0FCA3E0FDA3E0FEA3E0FF90FBA5
:1089A200B7E0F8A3E0F9A3E0FAA3E022121E0990CF
:1089B200FD12E0FCA3E0FDA3E0FEA3E0FF227E00A7
:1089C2007F407D0090FBADE0FBA3E0FAA3E022EB49
:1089D2002FFFEA3EFEE93DFDE83CFC22F9A3E0540C
:1089E2000F75F004A4F58285F08322EF4BFFEE4A67
:1089F200FEED49FDEC48FC226FFFEA6EFEE96DFDDB
:108A0200E86CFC225FFFEA5EFEE95DFDE85CFC22A9
:108A120090FD0EC9F0A3EAF0A3E9F07B017AFB799D
:108A22009622EF6BFFEE6AFEED69FDEC68FC229088
:108A3200FD12021E09121D7690FD0B22F074982B76
:108A4200F58274FB3AF5832274972BF58274FB3A14
:0D8A5200F58322F912227BE490FBAAF022AA
:10AAD80090FB96121E156745230190FB9A121E15CE
:10AAE800EFCDAB8990FB9E121E1598BADCFE90FB49
:10AAF800A2121E151032547690FBA6121E15C3D250
:0DAB0800E1F01289C0128A55A3F0A3F022DB
:1092BC0090FE65EBF0A3EAF0A3E9F0A3EDF0FF90CC
:1092CC00FBACE02FF090FBABE03400F090FE68E0DC
:1092DC00FF700302936290FBAAE0FEC374409EFEF3
:1092EC00C39F5004AF06800590FE68E0FF90FBB072
:1092FC00EFF07E001289C6F990FBAAE0FD7C00E934
:10930C002DF9EC3AA801FCAD0390FE651289C9F960
:10931C0012193990FBB0E0FF90FBAAE02FF090FE01
:10932C0066E48FF0121A9890FE68E0FF90FBB0E0B4
:10933C00FEC3EF9E90FE68F090FBAAE0C394404001
:10934C008B90FBAD1289A6128A12125F991289C0FA
:07935C00128A550292D8228B
:108556001289C6F990FBAAE0FF04F08F82758300AA
:1085660074801219D990FBAAE0FFC374409FC3948C
:108576000250071289C0F912227B90FBABE0FEA3E2
:10858600E07803C333CE33CED8F9F0EE90FBABF0F0
:10859600E0FF1289C6F990003EEF1219D990FBACA4
:1085A600E090003F1219D990FBAD1289A6128A12EB
:1085B600125F99E490FBB1F0A3F0C390FBB2E09494
:1085C6001490FBB1E0648094805066E0FEA3E0FF67
:1085D6002496F58274FB3EF583E0FD90FF80F074EF
:1085E600992FF58274FB3EF583E0FF90FBB1E0FA2C
:1085F600A3E0FB2496F58274FB3AF583EFF07499B9
:108606002BF58274FB3AF583EDF0128A4AE0FF906F
:10861600FF80128A3EE0FE128A4AEE128A3EEFF090
:1086260090FBB2E02404F090FBB1E03400F0028548
:05863600C0128A1D22A4
:105F990090FD0BEBF0A3EAF0A3E9F0121D2690FBAC
:105FA900B3121E09900004121D4690FBB7121E0978
:105FB900900008121D4690FBBB121E0990000C129E
:105FC9001D4690FBBF121E09900010121D4690FB42
:105FD900C3121E09E490FD11F090FD11E0FFD39466
:105FE9004F4003026285EFC3941050030260819011
:105FF900FD0E1289C9F9A3E024081289E1121D4690
:10600900C00790FD0EA3A3A3E0240D1289E1121D80
:10601900CDD007EB1289FAC00790FD0E1289C9F994
:10602900A3E024021289E1121DCDD007128A24C0EF
:106039000790FD0E1289C91289DE121DCDD00712F3
:106049008A2490FD121289AE7801121D13C004C072
:1060590005C006C0071289B1781F121CECD003D005
:1060690002D001D0001289EDC00790FD0E1289C936
:106079001289DED007121D9090FD0E1289C912896E
:10608900DE121D46128A3190FD121289A3FBC0004F
:10609900C001C002C00390FBB31289B47805121D78
:1060A90013C004C005C006C00790FBB31289B478B9
:1060B9001B121CECD003D002D001D0001289EDD004
:1060C90003D002D001D0001289D1128A3190FD117A
:1060D900E0D394135048A31289A3FBC000C001C0A8
:1060E90002C00390FBB71289B4121CDF90FBBF12E8
:1060F90089A3128A06C004C005C006AB071289929B
:10610900128A06D002D001D0001289EDEF2499FF3E
:10611900EE3479FEED3482FDEC345A02620390FDCF
:1061290011E0D39427502EA31289A3FBC000C0010C
:10613900C002C0031289921289FA90FBBF1289A387
:106149001289FAEF24A1FFEE34EBFEED34D9FDEC10
:10615900346E02620390FD11E0D3943B506FA31299
:1061690089A3FBC000C001C002C00390FBBF128914
:1061790095128A06C004C005C006AB07A31289B4EC
:1061890090FBB7A3A3A3E0128A06D002D001D000E6
:106199001289EDC004C005C006AB0790FBBF128988
:1061A900B490FBBB1289A3128A06D002D001D00099
:1061B900EB4FFFEA4EFEE94DFDE84CFCEF24DCFF16
:1061C900EE34BCFEED341BFDEC348F802D90FD12B6
:1061D9001289A3FBC000C001C002C0031289921238
:1061E90089FA90FBBF1289A31289FAEF24D6FFEE30
:1061F90034C1FEED3462FDEC34CAFCD003D002D0C8
:1062090001D0001289D1128A311289B190FBC312CF
:1062190089A3FBEF2BFFEE3AFEED39FDEC38FC12BA
:106229008A3190FBBF1289B4A3121E0990FBBB12DD
:1062390089B4A3121E0990FBB71289B4781E121DE6
:1062490013C004C005C006C00790FBB71289B47813
:1062590002121CECD003D002D001D0001289EDA3A8
:10626900121E0990FBB31289B4A31289AE90FBB335
:10627900121E0990FD11E004F0025FE290FD0B127D
:1062890089C9F9C002C001121D2690FBB31289A366
:106299001289D2D001D002128A371289C92404F98D
:1062A900E43AFAC002C001121D261289A01289D24D
:1062B900D001D002128A371289C92408F9E43AFABE
:1062C900C002C001121D2690FBBB1289A31289D2FC
:1062D900D001D002128A371289C9240CF9E43AFA9A
:1062E900C002C001121D2690FBBF1289A31289D2D8
:1062F900D001D002128A371289C92410F9E43AFA76
:10630900C002C001121D2690FBC31289A31289D2B3
:07631900D001D002021D7645
:03000000029B322E
:0C9B3200787FE4F6D8FD75816E029B7907
:10186900E709F608DFFA8046E709F208DFFA803E61
:1018790088828C83E709F0A3DFFA8032E309F6084E
:10188900DFFA8078E309F208DFFA807088828C83B6
:10189900E309F0A3DFFA806489828A83E0A3F6086A
:1018A900DFFA805889828A83E0A3F208DFFA804C44
:1018B90080D280FA80C680D4806980F2803380101B
:1018C90080A680EA809A80A880DA80E280CA803384
:1018D90089828A83ECFAE493A3C8C582C8CCC583FC
:1018E900CCF0A3C8C582C8CCC583CCDFE9DEE780CC
:1018F9000D89828A83E493A3F608DFF9ECFAA9F04B
:10190900EDFB2289828A83ECFAE0A3C8C582C8CCA0
:10191900C583CCF0A3C8C582C8CCC583CCDFEADEB9
:10192900E880DB89828A83E493A3F208DFF980CC1B
:1019390088F0EF60010E4E60C388F0ED2402B40414
:101949000050B9F582EB2402B4040050AF232345BB
:0619590082239018B9730F
:10195F00BB010689828A83E0225002E722BBFE0286
:09196F00E32289828A83E49322B9
:10197800BB010CE58229F582E5833AF583E0225024
:1019880006E92582F8E622BBFE06E92582F8E2226E
:0D199800E58229F582E5833AF583E4932288
:1019A500BB010989828A83F8E028F022500327F7D2
:1019B50022BBFE05F8E328F3228A838982F8E493A3
:0219C5002822D6
:1019C700BB010689828A83F0225002F722BBFE01FF
:0219D700F322F9
:1019D900F8BB010DE58229F582E5833AF583E8F044
:1019E900225006E92582C8F622BBFE05E92582C8F0
:0219F900F222D8
:1019FB00EF8DF0A4A8F0CF8CF0A428CE8DF0A42E00
:021A0B00FE22B9
:101A0D00BC000BBE0029EF8DF084FFADF022E4CCBD
:101A1D00F875F008EF2FFFEE33FEEC33FCEE9DEC86
:101A2D00984005FCEE9DFE0FD5F0E9E4CEFD22EDCC
:101A3D00F8F5F0EE8420D21CFEADF075F008EF2F16
:101A4D00FFED33FD4007985006D5F0F222C398FD07
:051A5D000FD5F0EA22A4
:101A6200C2D5EC30E709B2D5E4C39DFDE49CFCEE9F
:101A720030E715B2D5E4C39FFFE49EFE121A0DC3F0
:101A8200E49DFDE49CFC8003121A0D30D507C3E4EB
:061A92009FFFE49EFE220E
:101A9800C5F0F8A3E028F0C5F0F8E58215827002D9
:061AA8001583E038F02276
:101AAE00A3F8E0C5F025F0F0E582158270021583EB
:061ABE00E0C838F0E82248
:101AC400BB0110E58229F582E5833AF583E0F5F060
:101AD400A3E0225009E92582F886F008E622BBFE3D
:101AE4000AE92582F8E2F5F008E222E5832AF58383
:081AF400E993F5F0A3E9932248
:101AFC00BB010FF8E58229F582E5833AF583E8020C
:101B0C001AAE5011C58229F808C5F026C6F5F01892
:101B1C00C58236C622BBFE15C58229F808E2C5F07F
:101B2C0025F0F218E2C5823582F2E58222E5832A9D
:0C1B3C00F583E993F5F0A3E993C5F022CE
:101B4800BB010DC58229C582C5833AC583021A988F
:101B58005011C58229F808E5F026F618F5F0E58257
:101B680036F622BBFE11C58229F808E225F0F5F009
:101B7800F218E23582F222F8E58229F582E5832A15
:0D1B8800F58374019325F0F5F0E493382205
:101B9500F8BB0111E58229F582E5833AF583E8F082
:101BA500E5F0A3F0225009E92582C8F608A6F0223F
:0D1BB500BBFE09E92582C8F2E5F008F22226
:101BC200E88FF0A4CC8BF0A42CFCE98EF0A42CFCC2
:101BD2008AF0EDA42CFCEA8EF0A4CDA8F08BF0A440
:101BE2002DCC3825F0FDE98FF0A42CCD35F0FCEB9F
:101BF2008EF0A4FEA9F0EB8FF0A4CFC5F02ECD3964
:0F1C0200FEE43CFCEAA42DCE35F0FDE43CFC22D0
:101C110075F008758200EF2FFFEE33FECD33CDCC8A
:101C210033CCC58233C5829BED9AEC99E58298400D
:101C31000CF582EE9BFEED9AFDEC99FC0FD5F0D6EA
:101C4100E4CEFBE4CDFAE4CCF9A88222B800C1B914
:101C51000059BA002DEC8BF084CFCECDFCE5F0CB52
:101C6100F97818EF2FFFEE33FEED33FDEC33FCEB8B
:101C710033FB10D703994004EB99FB0FD8E5E4F946
:101C8100FA227818EF2FFFEE33FEED33FDEC33FC33
:101C9100C933C910D7059BE99A4007EC9BFCE99A27
:101CA100F90FD8E0E4C9FAE4CCFB2275F010EF2F6C
:101CB100FFEE33FEED33FDCC33CCC833C810D7076C
:101CC1009BEC9AE899400AED9BFDEC9AFCE899F8A7
:0E1CD1000FD5F0DAE4CDFBE4CCFAE4C8F9223A
:10A8D800C2D5E830E70FB2D5E4C39BFBE49AFAE4AB
:10A8E80099F9E498F8EC30E717B2D512A90E121CC2
:10A8F8004DE4C39BFBE49AFAE499F9E498F88003E1
:10A90800121C4D30D50DE4C39FFFE49EFEE49DFD6F
:04A91800E49CFC229D
:0D1CDF00CFF4CFCEF4CECDF4CDCCF4CC229A
:101CEC00E8600FECC313FCED13FDEE13FEEF13FFD6
:031CFC00D8F122FA
:101CFF00E86010ECA2E713FCED13FDEE13FEEF13FB
:041D0F00FFD8F022E7
:101D1300E8600FEFC333FFEE33FEED33FDEC33FC2E
:031D2300D8F122D2
:101D2600BB010789828A830222D45005E9F8021D85
:101D3600B4BBFE05E9F80222E089828A830222EC1E
:101D4600BB010DE58229F582E5833AF5830222D4AB
:101D56005007E92582F8021DB4BBFE07E92582F883
:101D66000222E0E58229F582E5833AF5830222EC38
:101D7600BB010789828A83021E095005E9F8021D04
:0A1D8600FDBBFE05E9F8022325224B
:101D9000BB010DE58229F582E5833AF583021E0930
:101DA0005007E92582F8021DFDBBFE07E92582F8F0
:041DB00002232522C3
:0C1DB400E6FC08E6FD08E6FE08E6FF225B
:0D1DC000E6FB08E6F908E6FA08E6CBF82293
:101DCD00BB010DE58229F582E5833AF5830222FCFC
:101DDD005007E92582F8021DC0BBFE07E92582F8F0
:101DED00022308E58229F582E5833AF5830223155E
:0C1DFD00ECF608EDF608EEF608EFF62212
:0C1E0900ECF0A3EDF0A3EEF0A3EFF0224C
:101E1500A8828583F0D083D082121E2C121E2C122C
:101E25001E2C121E2CE473E493A3C583C5F0C58351
:101E3500C8C582C8F0A3C583C5F0C583C8C582C817
:011E4500227A
:101E4600BB010DE58229F582E5833AF5830223433A
:101E56005007E92582F8022331BBFE07E92582F8FF
:101E6600022383E58229F582E5833AF583022395E9
:101E7600BB0120E58229F582E5833AF583D0F0D0CF
:101E8600E0F8D0E0F9D0E0FAD0E0FBE8C0E0C0F03E
:101E960002237A5018E92582F8D083D082D0E0F95F
:101EA600D0E0FAD0E0FBC082C08302233ABBFE1822
:101EB600E92582F8D083D082D0E0F9D0E0FAD0E0EC
:091EC600FBC082C08302238C22C0
:101ECF00D083D082F8E4937012740193700DA3A3A2
:101EDF0093F8740193F5828883E4737402936860B6
:061EEF00EFA3A3A380DFB6
:061EF5008A838982E47378
:101EFB00E5132582F582E5123583F583B51204854A
:101F0B0082132210AF06858213F51222858213F5F8
:041F1B0012D2AF220D
:0D1F1F00E5132582F582E5123583F5832256
:10A76B0090FE691222D47810EC4D4E4F70047CA5EC
:10A77B007DA5C3EC13FCED13FDEE13FEEF13FF50A1
:10A78B0010EC64CCFCED644CFDEE644EFEEF64CE3D
:10A79B00FFD8DF90FE69121E09EE547FFE2290FE59
:0DA7AB0069EEF0EFA3F0A374A5F0A3F02277
:10668500E508302C0104F8232824F8F582E434FBCE
:10669500F5832290FBF5302C0390FBF8E475F001AF
:1066A50012234C02195F60EAC50C7002150B14C564
:1066B5000C202C04FF02B64390FBF574FFF5F002A5
:1066C5002363FF02B4DCE5096006D509037F0022D8
:1066D500202C0F12B4C8EF6008050CE50C700205FC
:1066E5000B2290FBF512234312195FFF60E890FB24
:1066F500F5E475F00112234C80DC1266D5EFC0E09D
:106705001266C7D0E040F3809DD22C8002C22C9047
:10671500FBF512237AE4F50AF508F50BF50C750976
:1067250000C22BC229C22AC22D126698FF7005AF7E
:106735000A7E0022B42530126698FF24D0B40A00E0
:10674500500C75F00AC509A42509F50980E924CF7F
:10675500B41A00EF5002C2E5026973D22A80D8D27A
:106765002980D4D22D80D0EF1266C750081266FF5B
:10677500EF600E80A9EFC0E01266D5D0E06F609E95
:10678500EF60741266AB80A71266D5EF6069E50904
:106795007007050980031266D5EF6014202D0E12CF
:1067A5006685E475F00112234CEF1219C7D509E689
:1067B500202D040508050A80BA1266CBEFC0E01249
:1067C50066C7D0E050041266ABE4FF202D0E1266BA
:1067D50085E475F00112234CEF1219C7EF70DA202A
:1067E5002D040508050A808BE50960020509126676
:1067F500FF1266CBEF70C6302C04E41266ABE50AD7
:1068050060030267347EFF7FFF22202D1174FFFC99
:10681500FDFEFF126685122343121D7605080267E9
:1068250023D0E080D27900800A791080067908802B
:1068350002790AD22EE50960020509E9C0E012666F
:10684500FFEF60DD1266D5BF2D04D22B8003BF2B71
:10685500091266FFEF60CA1266CBD0E0B40A028067
:1068650033B40802802EBF302770027408C22EC0D0
:10687500E01266CBD0E0BF78028003BF5816050949
:10688500D509028007D50904D22E800B7410801912
:106895007002740ABF000AEFF8E4FCFDFEFF02690E
:1068A50026C0E0EF1266ABD0E0F9E4FCFDFEFFE99F
:1068B500C0E0ECC0E0EDC0E0EEC0E0EFC0E0126685
:1068C500CBEFF8D0E0FFD0E0FED0E0FDD0E0FCD08B
:1068D500F0E8604DB461004007B47B005002C2E5AA
:1068E50024D0503DFA24F6500724F95034240AFAEE
:1068F500EAB5F000502BCFA9F0A42FFF92D5E9C53A
:10690500F0CEA4A2D53EFE92D5E9C5F0CDA4A2D580
:106915003DFD92D5E9C5F0CCA4A2D53CFCC22E80A4
:066925008EE8C0E0202D09
:10692B002A202E08050A302B031222C61266851266
:10693B002343050820290B202A0DEE8FF01222A7E6
:10694B008009121D768004EF1219C7D0E01266ABD6
:10695B00026723202D101266851223430508E50BD1
:10696B00850CF01222A780E8121ECF67ED53682E1C
:10697B005867644C676042673C4868324F683644DE
:10698B00678D43682A49683655680F46680F456816
:0C699B000F4767682A695E4E0000676CB9
:101F2C00E3F5F009E208B5F06D606B80F3E3F5F0D2
:101F3C0009E608B5F060605E80F387F009E608B545
:101F4C00F054605280F487F009E208B5F04860461E
:101F5C0080F488828C8387F009E0A3B5F038603672
:101F6C0080F488828C8387F009E493A3B5F0276012
:101F7C002580F388828C83E3F5F009E0A3B5F01695
:101F8C00601480F388828C83E3F5F009E493A3B5A5
:101F9C00F004600280F2022057808580E7808E80FA
:101FAC00D2803C8015806C807E809B80B5808B803D
:101FBC00A1804F8070803A02206D89828A83ECFA6E
:101FCC00E493F5F0A3C8C582C8CCC583CCE493A335
:101FDC00C8C582C8CCC583CCB5F070606E80E18971
:101FEC00828A83E493F5F0A3E208B5F05E605C802E
:101FFC00F289828A83E0F5F0A3E608B5F04D604BD8
:10200C0080F389828A83E0F5F0A3E208B5F03C60A6
:10201C003A80F389828A83E493F5F0A3E608B5F05D
:10202C002A602880F2805D89828A83ECFAE493F539
:10203C00F0A3C8C582C8CCC583CCE0A3C8C582C8F0
:10204C00CCC583CCB5F004600280E27F00F845F08B
:10205C00600EE863F0806480D395F01F40027F012E
:10206C002289828A83ECFAE0F5F0A3C8C582C8CC39
:10207C00C583CCE0A3C8C582C8CCC583CCB5F0CB96
:10208C0060C980E389828A83ECFAE0F5F0A3C8C5C5
:10209C0082C8CCC583CCE493A3C8C582C8CCC58305
:1020AC00CCB5F0A760A580E288F0ED2402B4040062
:1020BC005099F582EB2402B40400508F23234582FF
:0520CC0023901FA57325
:10B49F00E4FFFE12195F600C0FEF70010E09E970E7
:05B4AF00F20A80EF220B
:1020D100E3F5F009E208B5F06BDFF58067E3F5F0B1
:1020E10009E608B5F05EDFF5805A87F009E608B524
:1020F100F052DFF6804E87F009E208B5F046DFF6D0
:10210100804288828C8387F009E0A3B5F036DFF640
:10211100803288828C8387F009E493A3B5F025DFB0
:10212100F5802188828C83E3F5F009E0A3B5F014F2
:10213100DFF5801088828C83E3F5F009E493A3B581
:10214100F002DFF4022200808780E9809080D48051
:102151003E8015806E807E809D80B7808D80A380BB
:10216100518074803C02220C89828A83ECFAE493C8
:10217100F5F0A3C8C582C8CCC583CCE493A3C8C578
:1021810082C8CCC583CCB5F076DFE3DEE18070890F
:10219100828A83E493F5F0A3E208B5F062DFF4806C
:1021A1005E89828A83E0F5F0A3E608B5F051DFF598
:1021B100804D89828A83E0F5F0A3E208B5F040DF23
:1021C100F5803C89828A83E493F5F0A3E608B5F0B3
:1021D1002EDFF4802A8002805789828A83ECFAE418
:1021E10093F5F0A3C8C582C8CCC583CCE0A3C8C50C
:1021F10082C8CCC583CCB5F006DFE4DEE280007F87
:10220100FFB5F0020F2240027F012289828A83EC0E
:10221100FAE0F5F0A3C8C582C8CCC583CCE0A3C859
:10222100C582C8CCC583CCB5F0D5DFE5DEE380CF70
:1022310089828A83ECFAE0F5F0A3C8C582C8CCC5CF
:1022410083CCE493A3C8C582C8CCC583CCB5F0AF19
:10225100DFE4DEE280A988F0EF60010E4E60ABEDB5
:102261002402B404005098F582EB2402B404005017
:0A2271008E23234582239021487339
:10227B00EF4E6012EF60010EEDBB010B89828A837A
:10228B00F0A3DFFCDEFA2289F05007F709DFFCA987
:0C229B00F022BBFEFCF309DFFCA9F022DE
:10A8030090FE16E0FFA3E0FEA3E0CF90FC51F0A37F
:10A81300EEF0A3EFF090FE19E0CBF0A3E0CAF0A3B3
:10A82300E0C9F07F2290FC54AD82AC8312195F8D96
:10A83300828C83F0A309E970010ADFEC90FE19E032
:0AA84300FBA3E0FAA3E0F90263852D
:109B3E00023DA5E493A3F8E493A34003F68001F25B
:109B4E0008DFF48029E493A3F85407240CC8C33328
:109B5E00C4540F4420C8834004F456800146F6DFF7
:109B6E00E4800B0102040810204080908E4BE47EAE
:109B7E00019360BCA3FF543F30E509541FFEE493EC
:109B8E00A360010ECF54C025E060A840B8E493A3B3
:109B9E00FAE493A3F8E493A3C8C582C8CAC583CADE
:109BAE00F0A3C8C582C8CAC583CADFE9DEE780BE96
:018F0E000062
:1022A700BB010A89828A83F0E5F0A3F0225006F782
:0F22B70009A7F01922BBFE06F3E5F009F319227F
:0E22C600C3E49FFFE49EFEE49DFDE49CFC2229
:0C22D400E0FCA3E0FDA3E0FEA3E0FF227D
:0C22E000E2FC08E2FD08E2FE08E2FF223A
:1022EC00E493FC740193FD740293FE740393FF2238
:0C22FC00E0F8A3E0F9A3E0FAA3E0FB2265
:0D230800E2FB08E2F908E2FA08E2CBF82255
:10231500E493F8740193F9740293FA740393FB221E
:0C232500ECF208EDF208EEF208EFF222F4
:09233100E6FB08E6FA08E6F922D1
:09233A00EBF608EAF608E9F622C8
:09234300E0FBA3E0FAA3E0F9229B
:10234C00F8E0FBA3A3E0F925F0F0E582158270021A
:07235C001583E0FA38F022BE
:10236300F8E0FBA3A3E025F0F9F0E5821582700203
:072373001583E038FAF022A7
:09237A00EBF0A3EAF0A3E9F02264
:09238300E2FB08E2FA08E2F9228B
:09238C00EBF208EAF208E9F22282
:0C239500E493FB740193FA740293F922A4
:10632000E50D2451F582E434FCF583E0050D22905F
:10633000FC4E30270390FC51E475F00112234C020F
:10634000195F2020E97F2ED2208018EF540F24906F
:10635000D43440D4FF30240BEF24BFB41A005003D0
:106360002461FFE50E6002150E0511E511700205AE
:106370001030270E90FC4EE475F00112234CEF0212
:1063800019C702B13F7403D2278003E4C227F50D79
:1063900090FC4E12237AE4F50EF510F511E50E602F
:1063A000077F2012636380F5750FFFC221C220C2F0
:1063B00022C223C225C226C22812632FFF700D30CD
:1063C00027057F00126374AF11AE1022B4255FC29F
:1063D000D5C22412632FFF24D0B40A00501A75F0DE
:1063E0000A780E30D50508B6FF0106C6A426F620A9
:1063F000D5047002D22380D924CFB41A00EF500400
:10640000C2E5D224026575D22180C6D22080C0D2D6
:106410002280BCD2D580BAD22580B47F201263639B
:106420002022077401B50E0040F1126320FF1263B1
:106430006302639DD228D2268095126320FB1263EB
:1064400020FA126320F94A4B700679467A667BFF80
:1064500020222EE50E602A7E008E8275830012199E
:106460007860060EEE650F70F0C2D5EBC0E0EAC0B2
:10647000E0E9C0E0EE1265BCD0E0F9D0E0FAD0E08F
:10648000FB12195FFF60AAEBC0E0EAC0E0E9C0E0E0
:10649000126363D0E02401F9D0E03400FAD0E0FBCD
:1064A000E50F0460DCD50FD980877BFF7A6579B86A
:1064B000D222809C791080027908C226C2288008E6
:1064C000D2D5790A8004790AC2D5E50F047002F5A5
:1064D0000FE4FAFDFEFF126320FC7B08202113125B
:1064E0006320FD7B1030200A126320FE126320FF20
:1064F0007B20EC3382D592D55013C3E43020069F25
:10650000FFE49EFEE42021039DFDE49CFCE4CBF827
:10651000C221EC700CCFCECDCCE824F8F870F3801B
:1065200017C3EF33FFEE33FEED33FDEC33FCEB33FB
:10653000FB994002FB0FD8E9EB302105F8D0E0C40D
:1065400048B221C0E00AEC4D4E4F78207B0070C26B
:10655000EAB50F0040BCC0E01265BED0F0D0E0202C
:106560002104C4C0E0C4B221C0F012634CD0F0D505
:10657000F0EB02639D121ECF643A5364B458640B6F
:106580004C64074264B84F64C04464C0496420430B
:0865900064C65564AA4664AA22
:106598004564AA47666650640F2D64132E64362B33
:1065A800641723643420664F2A63CF480000642EA2
:1065B8003F3F3F00790AA2D5202314302509B9109E
:1065C800020404B9080104A2D520260250010420BF
:1065D80022689222B50E005034C0E07F2030231983
:1065E8007F30A22272267225500F126615C222C26F
:1065F80026C225C2287F30800F302503E9C0E0126B
:106608006363302503D0E0F9D0E0B50ECC30251710
:106618007F30B9100C1263637F583024077F78806D
:1066280003B908031263633022057F2D0263637F79
:10663800202028F87F2B2026F322922280CF286E54
:10664800756C6C2900D2211263203021F8C22178A0
:106658000E30D50108F60263CF2D50434958126316
:10666800202403B405004001E4906661931263544A
:0D667800743A126354D223750E040264B408
:10B4C80010330B12B629BF0D027F0A02B13F90FE5E
:04B4D800FAE0FF2275
:08B6430090FEFAEFF0D2332271
:10B4DC00EFC394094005EF940E4004EFB42003D35E
:04B4EC008001C322F6
:10B13F00EFB40A07740D12B14A740A309811A89926
:10B14F00B8130CC2983098FDA899C298B811F63070
:07B15F0099FDC299F5992248
:0AB629003098FDAF99C2987E002210
:00000001FF
